:020000041001E9
:1000000000300030CF2C01107D2C01107D2C011010
:1000100000000000000000000000000000000000E0
:100020000000000000000000000000007D2C011016
:1000300000000000000000007D2C01107D2C01104C
:100040007D2C01107D2C01107D2C01107D2C0110C8
:100050007D2C01107D2C01107D2C01107D2C0110B8
:100060007D2C01107D2C01107D2C01107D2C0110A8
:100070007D2C01107D2C01107D2C01107D2C011098
:100080007D2C01107D2C01107D2C01107D2C011088
:100090007D2C01107D2C01107D2C01107D2C011078
:1000A0007D2C01107D2C01107D2C01107D2C011068
:1000B0007D2C01107D2C01107D2C01107D2C011058
:1000C0007D2C01107D2C01107D2C01107D2C011048
:1000D0007D2C01107D2C01107D2C01107D2C011038
:1000E0007D2C01107D2C01107D2C01107D2C011028
:1000F0007D2C01107D2C01107D2C01107D2C011018
:100100007D2C01107D2C01107D2C01107D2C011007
:100110007D2C01107D2C01107D2C01107D2C0110F7
:100120007D2C01107D2C01107D2C01107D2C0110E7
:100130007D2C01107D2C01107D2C01107D2C0110D7
:100140007D2C01107D2C01107D2C01107D2C0110C7
:100150007D2C01107D2C01107D2C01107D2C0110B7
:100160007D2C01107D2C01107D2C01107D2C0110A7
:100170007D2C01107D2C01107D2C01107D2C011097
:100180007D2C01107D2C01107D2C01107D2C011087
:100190007D2C01107D2C01107D2C01107D2C011077
:1001A0007D2C01107D2C01107D2C01107D2C011067
:1001B0007D2C01107D2C01107D2C01107D2C011057
:1001C0007D2C01107D2C01107D2C01107D2C011047
:1001D0007D2C01107D2C011000F002F800F0B5F824
:1001E0000CA030C8083824182D18671EA246AB464C
:1001F00054465D46AC4201D100F0A7F87E460F3E62
:10020000B6460FCC0126334200D0FB1A3343A24638
:10021000AB461847008B0000208B00000023002411
:1002200000250026103A01D378C1FBD8520700D32D
:1002300030C100D50B60704710B56E2902D100F0B7
:100240008CFE10BD702902D100F0A9FA10BD6629FC
:1002500002D107F04FFB10BD652902D107F04AFB20
:1002600010BD672902D107F045FB10BD612902D1FD
:1002700007F048FB10BD03681B0A01D38023194314
:10028000692902D100F016FA10BD642902D100F0EC
:1002900011FA10BD752902D100F00CFA10BD6F29BA
:1002A00002D100F075FF10BD782902D100F064FA88
:1002B00010BDE92902D100F011FF10BDE42902D1DF
:1002C00000F00CFF10BDF52902D100F007FF10BDB2
:1002D000EF2902D100F068FF10BDF82902D100F02B
:1002E00059FA10BD0368DB0901D380231943632940
:1002F00002D100F075FE10BD732902D100F078FE26
:1003000010BDE32902D101F056FE10BDF32902D140
:1003100001F059FE10BD002010BD1FB500980199D5
:1003200000F07DFD01F080FE04000020002107F0B8
:10033000B5FA401C60600020002107F0C5FAE060BB
:1003400001F0F8F800F03AFD1FBD0648854603B4F9
:1003500005F05AF903BC02F069FA02F07BFA05F0E5
:1003600093FC00000030003070B505460C46164680
:1003700002E00FCC0FC5103E102EFAD2082E02D389
:1003800003CC03C5083E042E07D301CC01C5361F9C
:1003900003E021782970641C6D1C761EF9D270BDB3
:1003A00070470000004870471433003070B50646AF
:1003B00000F018FD056830460B30C408E400B44274
:1003C00001D8002070BD68682A46002818D001684E
:1003D000A14211D30B46214608318B4208D3436812
:1003E00001194B6003681B1B0B605160046001E046
:1003F00041685160001D70BD024640680028E6D18A
:100400002146284600F0F6FC0028DCD170BD70B50E
:100410000446051F00F0E6FC0068002C1AD0446872
:1004200001E020466468002C01D0AC42F9D3016899
:100430000A18AA4204D12A6805468918016000E01A
:10044000456028684119A14205D161686960216849
:100450004018286070BD6C6070BD10B5202A04DBA8
:100460000146203A9140002010BD914020239C1A63
:100470000346E3401943904010BD10B5202A04DB29
:100480000846203AD040002110BD0B462024D3401E
:10049000D040A21A91400843194610BD434351432E
:1004A00030B55C18010C130C0D4692B25D4380B25E
:1004B00051432C19054655430A0C09044D19624154
:1004C0005843010C00044019514130BDFEB50546AA
:1004D00010460C46184373D0AE468C460020AD1A29
:1004E00001469C4167D36646002701243D46B61A63
:1004F0009D4102D313463A462124654676462F0491
:10050000360C3E432D0CB61A9D4104D3150C1B042A
:100510002B4312041034654676462F06360A3E43B6
:100520002D0AB61A9D4104D3150E1B022B4312024D
:100530000834654676462F0736093E432D09B61A1C
:100540009D4104D3150F1B012B431201241D654649
:100550007646AF07B6083E43AD08B61A9D4104D3B0
:10056000950F9B002B439200A41C65467646EF072F
:1005700076083E436D08B61A9D411AD392185B4126
:10058000641C16E00018764665464941B71A9D413D
:100590000191009009D36046B11A98418E46844675
:1005A000009801990025401C6941DD0752082A4343
:1005B0005B08641EE6D57246634603B0F0BDFFE7F4
:1005C00000200146C046C0462A462346F5E710B53E
:1005D0000B460146184600F00FFD10BD7CB51D46C8
:1005E00016460C00009001D00019401E084B7B44B9
:1005F0002A4669460190304600F0C7FC002C0546AB
:1006000003D06946002000F0D3FC28467CBD0000E2
:10061000C909000070B5044685690068C10601D5A6
:10062000302600E02026C00707D070BD6268304643
:10063000A1689047206A401C20626D1EF6D570BDEF
:1006400070B5044685690078C00707D170BD62683F
:10065000A16820209047206A401C20626D1EF6D5BC
:1006600070BD70B50C460546012A05D02878800675
:1006700000D5EA69002302E0012305E05B1C9342F8
:1006800002D2E05C0028F9D1A869E618C01AA86176
:10069000286AC01828622846FFF7BCFF04E06A6891
:1006A0002078A968641C9047B442F8D32846FFF725
:1006B000C7FF70BDF7B5002575291068009914A60D
:1006C00011D000F0E0FB002802DA404211A608E059
:1006D000009909688A0701D50FA602E0490704D5E9
:1006E0000EA6012501E000F0D7FB009F002424376F
:1006F00004E001F06AF830313955641C0028F8D163
:100700002B4632462146009800F0CFFBFEBD00008C
:10071000000000002D0000002B0000002000000061
:10072000F8B50F460188090502D5224C7C4402E049
:10073000204C7C440E3405460021243508E0160781
:100740001209360FA65D6E541E0732431B09491C61
:1007500016461E43F3D1224604780023240705D50C
:10076000702F06D0002901D00223113200F09DFB2A
:10077000F8BD01231032F9E770B504460D46214655
:10078000106800F089FB0023024629462046FFF747
:10079000C7FF70BDD21DD308DB000CCBC0E730B45F
:1007A000036820241268234303600823C36130BC1C
:1007B0000023B5E7E4710000F3B50446002081B0E2
:1007C00020622046E1688847002872D0252802D0A0
:1007D0006268A168ABE0594F00267F442046E1687B
:1007E00088472028054608DB312D06D278192038A5
:1007F0000078002801D00643F0E7B00701D50420B7
:1008000086430020E0610746A0612A2D0AD02846D1
:1008100007F02EF8002827D0B8000019303D0090CE
:10082000856119E00298BA00121902C8916102901C
:100830002046E1688847012F054617D1E069002866
:100840001FDA202086431CE000980A218069484373
:1008500000994019303888612046E168884705468C
:1008600007F006F80028EFD1012F0AD02E2D08D16D
:100870002046E16888470546202006437F1C022F5A
:10088000C3DBA069002803DA4042A06101200643CF
:10089000F00701D0102086436C2D0BD0682D09D0B5
:1008A0004C2D3CD06A2D38D0742D38D07A2D36D0CE
:1008B00016E040E0E1682F4620468847B8420546EA
:1008C00009D16C2F29D001208002E168064320461F
:1008D0008847054604E06C2F1DD0FF2001300643F9
:1008E000002D28D028464138192803D80120C002FD
:1008F00006432035204626602946029A1646FFF711
:100900009BFC002810D001280BD0F61DF008C00079
:100910000830029055E74020E1E78020D5E700202D
:10092000D3E7361D02964CE762682846A1689047D7
:10093000206A401C44E7206AFEBD00005E71000092
:10094000F8B5044616460D464769007B800730D04F
:10095000384604F080FE00282BD132461026002AAB
:1009600025D0012A02D0022A23D104E0204600F03B
:1009700021FD45191BE0384604F05BFEE168314378
:100980000028E16004DA204600F05CFD0120F8BD9B
:10099000C9030BD56268E16A914200D81146A26989
:1009A00089182269891A814200DD08462D18002D18
:1009B00001DA0220F8BDE16A6068E268814206D28D
:1009C0009103E06203D5012149048A433243A669B9
:1009D000AE4211DCE16A814201D90B4600E00346D8
:1009E0009F192369FF1AAF4206DD814201D90F46E4
:1009F00000E007469F4206D1202002430020A0606D
:100A0000A56220600DE0AD1BE669AE1B8142A660C9
:100A100000D90846C01A281A2060581960602020A2
:100A20008243034802400020E26040342072F8BD57
:100A3000BFCFD7FFF7B516460C46104600F06EF84C
:100A40002078611C61280AD0722802D0772839D119
:100A500002E00125002404E00225042401E02D4DDC
:100A600008240222032301270878491C2B2806D0DA
:100A7000622807D02039C87F742807D008E01D43BA
:100A80001443F1E7042005433C43EDE71020044301
:100A90000098214604F0E2FD411C13D00021316191
:100AA00071600121F5604902F1617061200704D590
:100AB000304602220021FFF743FF306D3843306596
:100AC0003046FEBD0020FEBDF8B50D460646124C70
:100AD000206DC10704D0410804D044086400F7E742
:100AE000224610E05420FFF761FC070010D079087F
:100AF000206D4900012211430843542120653846E6
:100B000000F011F93A4629463046FFF793FFF8BD49
:100B10000020F8BD0280000018330030FEB5044606
:100B2000466900690F4F0190E56800200090A80712
:100B300007D0204600F0B6FC304604F077FD0028D0
:100B400001DA3846FEBD280502D50198FFF75FFCA3
:100B50004C21204600F0E7F8206D40084000206559
:100B60000098FEBDFFFFFFFF30B503461D78002D46
:100B700008D00A461478521C002C03D0AC42F9D19C
:100B80005B1CF3E7181A30BD034610B50B439B07F7
:100B90000FD1042A0DD308C810C9121FA342F8D0E0
:100BA00018BA21BA884201D9012010BD0020C043E3
:100BB00010BD002A03D0D30703D0521C07E0002049
:100BC00010BD03780C78401C491C1B1B07D103780F
:100BD0000C78401C491C1B1B01D1921EF1D11846F8
:100BE00010BD000030B5441C03E00178401C002912
:100BF0000DD08107F9D10B4BDD0104C8D11A914307
:100C00002940FAD0001B0A0603D0C01E30BD001BCD
:100C100030BD0A0401D0801E30BD0902FCD0401E48
:100C200030BD000001010101F8B5042A2CD383076F
:100C300012D00B78491C0370401C521E83070BD046
:100C40000B78491C0370401C521E830704D00B789C
:100C5000491C0370401C521E8B079B0F05D0C91AFC
:100C6000DF002023DE1B08C90AE0FFF77DFBF8BD8B
:100C70001D4608C9FD401C46B4402C4310C0121F3D
:100C8000042AF5D2F308C91A521EF0D40B78491C75
:100C90000370401C521EEAD40B78491C0370401CA0
:100CA000012AE4D409780170F8BD134610B5044652
:100CB000CAB219461002821810048218204600F0A9
:100CC00021F8204610BDD2B210B513029A181304B1
:100CD0009A1800F017F810BDD2B210B513029A1886
:100CE00013049A1800F001F810BD01E004C0091FB8
:100CF0000429FBD28B0701D50280801CC90700D0D4
:100D00000270704700290BD0C30702D00270401C4C
:100D1000491E022904D3830702D50280801C891E44
:100D2000E3E70022EEE70022DFE70000024670B5AD
:100D30000A4392072AD11E4DEE0104C808C9541B6C
:100D40009443344017D0D0B2D9B2401A210601439F
:100D500010D190B299B2401A210401430AD1100275
:100D60001902000A090A401A2102014302D1100E99
:100D7000190E401A70BD9A42DFD010BA19BA8842D3
:100D800001D9012070BD0020C04370BD02780B78EE
:100D9000401C491C002A09D09A4207D102780B78DE
:100DA000401C491C002A01D09A42EFD0D01A70BDD5
:100DB00001010101704770477047000070B5064C93
:100DC0007C44064D7D4403E0206800198047241DC3
:100DD000AC42F9D170BD00009C8000009C800000F6
:100DE0007047000000487047143400307047704767
:100DF0007047704738B504460A4600206946C04629
:100E0000C046002805D002462046009900F0FAFCB2
:100E1000012038BD10B5012001F000F910BDF8B572
:100E2000C046C046054600200C461020C046064677
:100E3000A819A0420DD9324669460020C046C046D6
:100E4000070001D101F0EAF80098A04200D0054661
:100E5000C419FFF7C7FFF61D07460560F008C0007C
:100E60004619284600F008F8B44204D031463868E4
:100E7000A21B00F0C7FCF8BD00210160416080604A
:100E800070471020704709684A0501D540B2704785
:100E9000C905FCD500B2704709684A0501D5C0B242
:100EA0007047C905FCD580B27047FFB504460D46B2
:100EB00081B0243000902168880604D51022E069B2
:100EC0009143216000E00120A84201DD471B00E0C2
:100ED00000270498A1697A191018081AA0612078CF
:100EE000C00602D42046FFF795FB002608E00398D1
:100EF0006268A168805D9047206A401C761C206271
:100F000004988642F3DB2078C0060AD52046FFF716
:100F100081FB06E06268A16830209047206A401C8F
:100F2000206238467F1E0028F4DC07E000986268E3
:100F3000A168405D9047206A401C206228466D1ED3
:100F40000028F3DC2046FFF77BFB2078000602D563
:100F5000022005B0F0BD0120FBE711680268006ABD
:100F6000530501D5087009E0D30501D5088005E0D7
:100F7000130602D5C21705C100E0086001207047C2
:100F800001694A1C02610878704700B58FB0029170
:100F9000002105910549019379440391114604907C
:100FA0006846FFF709FC0FB000BD0000E5FFFFFF3A
:100FB0000A681070521C0A6070470CC908399A42BE
:100FC00002D2531C0B601070704710B54369002BA0
:100FD00002D0C046C04601E0FFF743FB012010BD30
:100FE0001278014624310A7000224A700122ECE78F
:100FF00011680022D243E8E7084B70B50D467B44E8
:10100000FFF7C3FF0446284600F0D8F8002802D0B6
:101010000020C04370BD204670BD00007D68000008
:10102000F7B50446154686B02B487844002703C818
:101030003E460090019111E007986A467100415ABE
:1010400002A800F0C4FF411C07D02178890603D50F
:10105000E269391891420ED83F18761C2078800634
:1010600002D5E069B84206DDAE42E5DB07987100C3
:10107000405A0028E0D1A069C01BA0612046FFF7BC
:10108000C9FA154878445A3803C8009000200191E5
:1010900016E041006A460798415A02A800F097FFFF
:1010A0000590401C0AD0002505E0626802A8A168EE
:1010B000405D90476D1C05988542F6D30498401C0E
:1010C000B0420490E5DB206AC01920622046FFF799
:1010D000B7FA09B0F0BD000022690000F7B5D21DD3
:1010E0000025D20815A6D200F52905CA11D0002A7C
:1010F00005DA00214042914111A60A4608E0009914
:1011000009688B0701D50FA602E0490701D50EA695
:1011100001251146009F0024243704E000F08CFBD9
:1011200030323A55641C02460A43F7D12B46324608
:1011300021460098FFF7B9FEFEBD00000000000048
:101140002D0000002B0000002000000070B50446B8
:101150000021243408E05507D2086D0F303565545E
:101160005D072A43DB08491C15461D43F3D104687B
:10117000002310A2250708D520252C400C4304D0BD
:10118000C46901230CA2641EC461FFF78EFE70BD0A
:1011900010B5044621461068FFF77EFE0023024684
:1011A0002046FFF7D3FF10BDD21DD108C9000CC9DE
:1011B000CCE700000000000030000000C068802183
:1011C00008407047F8B505460C46C8680521C904B3
:1011D0008843012189050843E060800602D5204646
:1011E00000F086F97149E0680140022903D02046E9
:1011F00000F028F9BCE00521012249030140D20397
:1012000091420FD1C00306D56168E06A884200D8D8
:101210000846606006E02069E0626060606904F092
:1012200008FAA061A1680022EEB200290EDAE06897
:1012300083050BD4C943A1600921226049030843F7
:10124000E0606068411C61600670ACE0E06801210C
:1012500049030843E060002020602069002831D164
:10126000606904F0F8F9012527462437ED020028CB
:1012700016D0A0898005800F08D0E069FFF796F8A6
:101280000028206102D0E068284318E0012027618F
:10129000E061E068032109028843012189020DE031
:1012A000E069FFF783F800282061EFD0E068284369
:1012B000E0608105890F03D1FF2101310843E0601F
:1012C00020696060E2683A4F2569D0051FD56168E2
:1012D000E06A884200D80846411B05D022462846CD
:1012E00000F0BAF8002843D1E068010204D5E562B5
:1012F00000206560A06053E0691CE1626160E16903
:10130000491E3843A160E06030462E70F8BD1002DF
:1013100001D53A4009E06068411C61600670E068F0
:1013200038430A2EE06006D00022E16A60688142FC
:1013300003D90B4602E00122F7E70346A7895B1BAE
:101340007F0504D4E7699F4201DD002A1ED0814257
:1013500000D801460F1A0020E5626560002BA060EE
:1013600009DD22461946284600F076F8002802D00A
:101370000020C043F8BD002F08D0A069E562656079
:10138000C01BA061E06810210843E060E068000233
:1013900009D56168A069E562491B40186560A061D4
:1013A0000120C043F8BD3046F8BD000082100000A7
:1013B0000000010010B50146C268900703D09006F6
:1013C00007D5886A0AE0FEF7EDFF01210160881E5B
:1013D00010BD8B694868C0180B69C01A40310B7A80
:1013E000002B02D0497A401A10BD1103FCD5002809
:1013F000FADD401E10BD000070B5C468A50713D00B
:10140000650211D4D51FF93D0AD0FF3D6D1E07D0EE
:10141000FF3DFF3D022D07D101462431012305E0A8
:10142000074E5D1EB54201D3012070BD0161C3614D
:1014300041600F2109028C431443C460002070BD39
:10144000FFFFFF00C1688022114392039143C160F6
:101450000021816001607047F7B514460E4633489D
:10146000D5685769054209D03846A16904F044F9A6
:10147000002811DB2D48C0430540E5602B4632466D
:101480003846009904F03BF94200A1695208B21AAB
:1014900089180028A16104D02046FFF7D3FF00205F
:1014A000C043FEBD70B504460569C06A61688842E4
:1014B00000D80846E1680522D2049143E160C903DF
:1014C00014D5A84209D02246411B2846FFF7C4FF85
:1014D000002802D00020C04370BDE5620020656096
:1014E000A060E068012109048843E060002070BD2D
:1014F00010B50446C06820218843E060A16AA06955
:1015000088420ED02046FFF7CDFFE0680321090393
:10151000884310210843E060A06AA0612069E0626E
:1015200060600349E0680840E06010BD1000020000
:10153000BFBFFFFF10B543485421FFF7F4FB4248FB
:101540005421FFF7F0FB41485421FFF7ECFB4048E2
:101550003C493D4B404A01603E4803603B481060B7
:101560005A1C0A65411C1965012101653C48354A30
:101570003AA17844FFF75EFA002804D1384878444D
:101580000C3800F045FD38482F4A36A17844FFF763
:1015900051FA002804D1344878440C3800F038FD62
:1015A00032482A4A2FA17844FFF744FA002804D190
:1015B0002E4878440C3800F02BFD40232148DC00F5
:1015C00000212246FFF718FF002804D02448784461
:1015D0005C3800F01DFD1C48224640230021FFF727
:1015E0000BFF002804D0204878445C3800F010FD40
:1015F0001648224610230021FFF7FEFE002804D0E3
:101600001A4878445C3800F003FD10BD0F4870B5EF
:10161000006D44080B486400FFF780FA0A48FFF7A2
:101620007DFA0A48FFF77AFA09E0206D450820465E
:101630006D00FFF773FA2046FEF7E9FE2C46002CFA
:10164000F3D170BD183300306C330030C03300303C
:10165000E0310030E4310030E83100307200000049
:10166000C270000077000000AF70000086700000BC
:10167000002203098B422CD3030A8B4211D300238F
:101680009C464EE003460B433CD4002243088B4269
:1016900031D303098B421CD3030A8B4201D39446F6
:1016A0003FE0C3098B4201D3CB01C01A52418309E9
:1016B0008B4201D38B01C01A524143098B4201D3A3
:1016C0004B01C01A524103098B4201D30B01C01ACE
:1016D0005241C3088B4201D3CB00C01A5241830848
:1016E0008B4201D38B00C01A524143088B4201D375
:1016F0004B00C01A5241411A00D2014652411046D5
:1017000070475DE0CA0F00D04942031000D3404249
:1017100053409C46002203098B422DD3030A8B427F
:1017200012D38901FC2212BA030A8B420CD389011D
:1017300092118B4208D3890192118B4204D3890103
:101740003AD0921100E08909C3098B4201D3CB0141
:10175000C01A524183098B4201D38B01C01A5241F6
:1017600043098B4201D34B01C01A524103098B42FA
:1017700001D30B01C01A5241C3088B4201D3CB00E5
:10178000C01A524183088B4201D38B00C01A5241C8
:10179000D9D243088B4201D34B00C01A5241411A9F
:1017A00000D201465241104663465B1001D34042CD
:1017B000002B00D54942704763465B1000D340427E
:1017C00001B50020C046C04602BD01468008081A87
:1017D00002091018020A1018020C1018C008820022
:1017E00012185200891A01E0401C0A390A29FBD25A
:1017F0007047000010B500F017FC001D10BD00BFC1
:101800009D60000010B50346406801E00346406853
:10181000002801D08842F9D31868C3188B4206D03B
:10182000CB1CD808C000001D411A521A0146081DE1
:101830000A60FEF7ECFD10BD0B4670B50246890745
:101840008008084319469D08141AA941250908076C
:10185000054308092C194841250A01060D43010AD0
:101860002C194141200C0D0428430D0C00194D4149
:10187000002140194D41C00869070843E908840F59
:101880008D002543840024184D4124196D41121BFD
:10189000AB4107E00925ED432C11521963410024A7
:1018A000401C61411C460A250026551BB441F1D25B
:1018B00070BD0000FFB50C461E468FB003CA0890ED
:1018C00009914F007D0D00D16D1E002108460020BA
:1018D000C0460321099A89050840002A03DA8200DC
:1018E000801840080840800D01280A9002DD002081
:1018F000C0430A90089807430DD0F048F0492818D3
:1019000048430714189800281DD07542291E1DDD74
:101910000A9842421BE01898012802D0002030218A
:1019200004E00020F24305E02154401CB042FBDB00
:1019300030460022189B002121540F998B600A60C9
:10194000486013B0F0BDBD1B6D1CDFE70A9A00298B
:1019500000DA69420BA800F0AFFB0BAB07CB03AB7F
:1019600007C30899099800F013FC6B4607C30146AA
:10197000D4480918002D00910BDDD24903980A9A2A
:1019800049424018002303A90390684600F070FE06
:1019900008E003990A9A0023081803A903906846EF
:1019A00000F010FE6B4607C30004000C03D00020BB
:1019B000C043410800E01046189A002A03D00022D4
:1019C000009215461EE0751E05D4FFF735FF303234
:1019D00062556D1EF9D501220843079602D00022F8
:1019E0007F1C04E02078302801D100227F1E002ACD
:1019F000069787D01EE0112D07DAFFF71DFF303262
:101A000062556D1C02460A43F5D1084303D0009885
:101A1000002819D00EE00021681E05E0235C625CFE
:101A200063542254401E491C8142F7DBA81B401E10
:101A300007950690079A18990020A0540F98079BC5
:101A4000069A81600CC07CE711260020189059E7A7
:101A5000D21DF0B50D460446D10893B0C90003C9A4
:101A60000C900D9105F0EEFE02460D98C00F01D0CE
:101A70002D2007E02068810701D52B2002E04007D8
:101A8000C00F4001032A0F9001D0072A05DB03464F
:101A90002946204600F0CCFA0EE12078800601D5D8
:101AA000E76900E006272846652D04D0662814D093
:101AB000672D69D12DE00020112F009001DB11234B
:101AC00000E07B1C0CAA03A910A8FFF7F3FE1199F4
:101AD000002610987D1C0E9142E001203B460CAA86
:101AE000C0070B900120009003A910A8FFF7E2FEA9
:101AF000119D12981099002600280E9501D1781C8E
:101B00000D18781B02D446427D1C761EE81B0090FF
:101B10003AE0012F00DA01270020112F009001DDAB
:101B2000112300E03B460CAA03A910A8FFF7C2FE50
:101B300011993D46109800260E91217809070BD483
:101B40000E99A94200DA0D4603A9012D04DD4A19B8
:101B5000203AD27F302A06D0B84201DA011D04DAD9
:101B6000012100910FE06D1EEFE7002802DC8619CD
:101B70002D1A03E0411CA94200DD0D46801B401CCC
:101B800000900120C0070B902078000705D4009832
:101B9000A84202DB0020C043009069460020C872C2
:101BA0000B98012102AF0337C907884225D00220D4
:101BB00010902B2011900B9800280BDA40420B90CC
:101BC0002D20119006E00B98FFF7FFFD30317F1EAE
:101BD0000B9039701099481E00291090F3DC0B9877
:101BE0000028F0D111987F1E38702088000501D59B
:101BF000452000E065207F1E387001A8C01BC01D75
:101C00000B900F98002800D0012041190098C017B0
:101C100009180B980818A169081A401EA0612078BD
:101C2000C00602D42046FEF7F5FC0F98002805D028
:101C30006268A1689047206A401C20622078C00634
:101C400025D52046FEF7E6FC21E0002E07DB0E98A6
:101C5000B04204DD03A86268805DA16802E06268AA
:101C6000A16830209047206A761C401C20620098B2
:101C7000401E002800900AD100F0D6F9C0686268C2
:101C80000168405CA1689047206A401C2062284699
:101C90006D1E0028D9DC07E062683878A1687F1CD7
:101CA0009047206A401C20620B99481E00290B9027
:101CB000F2DC2046FEF7C4FC032042E601FCFFFFF5
:101CC000104D0000E1DFFFFFD21DF0B504460D46C8
:101CD000D0088DB0C000466807683146384605F028
:101CE000B1FD0246F00F01D02D2307E020688107E7
:101CF00001D52B2302E04007C00F43016846002BAB
:101D0000037001D0012000E00020032A0A9001D0D6
:101D1000072A04DB2946204600F08AF92DE12078C5
:101D2000800601D40D2500E0E5697000400D0D2D01
:101D300001904BDA300D00210B9008460020C04680
:101D4000032189050840002E05DA82008018C20FA1
:101D50001018401008408015012801DD0020C04304
:101D6000A9000023182906D39C460A460123183AE5
:101D70001B07D34003E001221205CA4094460C31F0
:101D8000202902D33A46203900E032468A40002812
:101D900002DD002A06D119E0002817D10121C90768
:101DA0008A4213D3194663467F185E41002806D144
:101DB0000120C007824202D1084687439E430B9808
:101DC000310D814202D00198401C0190208800050D
:101DD00002D57149794402E06F49794419396B465B
:101DE0000A9830221A540A980A7C401C1A54401C43
:101DF0000A900198002801DC302000E031201872A0
:101E0000019A0120002A02D0644BD21804E072002B
:101E10003A4302D0614A521C0192002D02DC227822
:101E2000120703D56A462E205072022000228646F1
:101E300094460CE032033601120F6D1E8B5C02AA31
:101E400013546246521C401C9446052A01DA002DA8
:101E5000F0DC002202AE08E03B0F3F01CB5C521CDD
:101E60006D1E3354401C082A01DA002DF4DC23686F
:101E70009A0601D511E0401E704504DD3218203A63
:101E8000D27F302AF7D0002807DD3218203AD27FDF
:101E90002E2A02D11A0700D4401E002D03DD3E2257
:101EA0003254401C6D1E497C31540199401C00295C
:101EB00006DA2D21471C315401984042019003E07D
:101EC0002B21471C315401987D21C900884206DB33
:101ED000FFF7D8FB3030F0557F1C019101E06428FA
:101EE00008DB01986421FFF7CDFB3030F0557F1CF3
:101EF000019101E00A2806DB01980A21FFF7C2FBE5
:101F00003030F0557F1C01980A21FFF7BBFB3031C0
:101F1000F1550A98A1697F1C7A191018081AA06156
:101F20002078C00602D42046FEF774FB216A6E4674
:101F30000A980818206204E062683078A168761C6C
:101F400090470A98401E0A90401CF5D12078C006A0
:101F500002D52046FEF75EFB02AE09E03078761C23
:101F60003E280DD06268A1689047206A401C20621C
:101F70007F1EF3D22046FEF763FB0DB00320F0BDB9
:101F8000206A4019206203E06268A168302090470F
:101F90006D1EEDD3F8E70000935B000001FCFFFF2E
:101FA00010B54369002B02D0C046C04601E0FFF7E0
:101FB00037F8012010BD12880146243182840022A6
:101FC000C2840122ECE711680022D243E8E7F8B5A9
:101FD00016460C460546FFF70DFC0368FF2002304D
:101FE000C05C012807D0FF2C0FD8185D00280CD04A
:101FF00001202C70F8BDFF333246214608331868A3
:10200000C71828460023B847F8BD0020C043F8BDD4
:1020100010B500F083FB00F07BFB10BD10B500F0A5
:1020200097FB00F075FB10BD004870471834003076
:10203000F8B51F46044601230068DB02032601466B
:102040001840072A05DB002801D017A506E017A5D0
:1020500004E0002801D016A500E016A51020814359
:102060002160A069C01E002FA06101D0401EA061A8
:102070002046FEF7CFFA002F09D038466268A168E3
:102080009047206A401C2062C01C206206E0206A43
:10209000FAE762682878A1686D1C9047761EF8D22E
:1020A0002046FEF7CDFAF8BD4E414E006E616E003F
:1020B000494E4600696E6600F7B516468AB0334849
:1020C00078446C4603467C33C06F5A689B680DC4E5
:1020D0002E487844763003AC0DC80DC43720C001BB
:1020E000081837211B30FFF7CDFA05460C46803D16
:1020F0001B3C02D56442012000E00020002709902B
:1021000010E0E0070CD00C20204978437944324697
:102110004C3941186846012300F054FA6B4607C356
:1021200064107F1C002CECD1184F7F442E3F16E02A
:10213000E80712D02001C0190EC806910893079233
:102140000068F04201D1981908903246012306A98F
:1021500003A800F037FA03AB07C36D10641C002D11
:10216000E6D10998002806D032466946012303A823
:1021700000F07EFA05E001233246694603A800F02C
:1021800021FA0A9B07C30DB0F0BD0000BC58000047
:10219000034640000A4610B5400D0BD00121C90787
:1021A0000F24A40200191C0364082143540D214389
:1021B000D20207E000210120F2E7D40F49002143B9
:1021C0005200401E0029F8DADB0FDB07184310BD70
:1021D000FFB50D46144685B04868516805F018FBF8
:1021E00000910190A868A16805F012FB029103908C
:1021F000A868616805F00CFB029A121882420292EC
:1022000001D2012000E00020019A0B18D21800280A
:10221000019202D08A4202D903E08A4201D201200F
:1022200000E000200099081800906868A16805F097
:10223000EFFA029A12188242029201D2012000E0C3
:102240000020019A0B18D2180028019202D08A426D
:1022500002D903E08A4201D2012000E00020009967
:102260000818009028682168400049004008490883
:102270004018FA49471814E001994000C90F084373
:102280000090019802994000C90F084301900298FC
:1022900003994000C90F08430290039840007F1E35
:1022A000039000980028E7DA0898002801D0EC4E47
:1022B00000E00026B74201DA012000E000200028FB
:1022C00004902AD0F71BF806C00E15D0029B2021DF
:1022D000091A039A8B401A430392029A019BC24047
:1022E0008B401A430292019A009BC2408B40009996
:1022F0001A430192C14000917B110DD06F4603201B
:10230000C11A03D500218200B95003E08A00810080
:10231000BA587A50401EF3D53746039802990028E0
:1023200000D00120014308980291002808460CD0F3
:10233000002800D001200199019A49050843012194
:10234000D20AC902D202019200E001210E9B0122B1
:10235000D207012B02D0002B03D013E0002807D1B5
:1023600020E0904204D890420CD1019B0B4209D04E
:10237000019B5918019105D10099491C009101D187
:102380007F1C009200280DD0102108460020C04676
:102390000498002806D00F98002803D0082108468A
:1023A0000020C04628682168019B009A4840C10F60
:1023B0000598C90739430EC009B0F0BDFFB587B015
:1023C000099A0898089953689268406889689646FF
:1023D0000022039317469446089A12685300099AFC
:1023E0005B081268520052089A1A9E4BD4180A9A37
:1023F000002A01D0352200E040220692002201236B
:1024000015460492DB07059324E0002D05D175469F
:102410000346039E4D1BB34109D375466646039B95
:10242000491B049D9841059B7519AC465F41634665
:102430003B4308D0059B049EDD0776082E435B08CE
:102440000496059301E0521E641EC50FED0749185E
:102450004041521C069B9A42D7DB002D04D17546A1
:10246000039A6B1A824101D203200CE0039A0B46B7
:102470006B404240134303D0014303D0012002E0EC
:10248000022000E0002061460191002100970291A6
:102490000A99002905D0614640020143704B019121
:1024A00002E08007002302909C4201DA012000E054
:1024B000002007003AD01A1BD006C00E15D0029D8E
:1024C0002021019C091AC5408C402543029C8C4068
:1024D00000D001242543019C0295009DC4408D40FD
:1024E00000992C430194C140009154111DD06D46B8
:1024F0000221002202290CD10320001B07E0002842
:1025000004DB8600AE59002E00D00122401C0328B7
:10251000F5DB081B02D588002A5004E0800028580B
:1025200010438A00A850491EE3D51C460A9800288B
:1025300002980CD0002800D001200199019A490589
:1025400008430121D20AC902D202019200E001210E
:10255000109B0122D207012B02D0002B03D013E0E5
:10256000002807D11FE0904204D890420CD1019B73
:102570000B4209D0019B5918019105D10099491CC2
:10258000009101D1641C009200280CD01021084653
:102590000020C046002F06D01198002803D0082143
:1025A00008460020C04608980999019A009B0068D7
:1025B00009684840C10F0798C907214382600AC0D3
:1025C0000BB0F0BD00B585B0019300920A460146FC
:1025D000002302A8FFF7FCFD02A807C805B000BD54
:1025E000FFB50A461F4685B0079901930123009164
:1025F000014602A8FFF7ECFD02990398049ECA0F5A
:102600004900D20700920F22490892028C1A002139
:10261000002800DB0C46450013486D08844214D3A3
:10262000079A002A04DA441E0026104DF64302E001
:1026300004460D460E46102108460020C046002FD5
:1026400003D0042108460020C0462005E90A0843BB
:10265000009908436905F20A1143ADE602C0FFFF85
:10266000013C0000FF3F0000FF070000FFFFFF7F6D
:1026700000B585B0019300920A460146002302A8E6
:10268000FFF79CFE02A807C8A8E7FFB50A461F4649
:1026900085B00799019301230091014602A8FFF735
:1026A0008DFE02990398049ECA0F4900D20700923A
:1026B0000F22490892028C1A0021002800DB0C46E8
:1026C000450011486D08844214D3079A002A04DAA1
:1026D000441E00260D4DF64302E004460D460E460C
:1026E000102108460020C046002F03D004210846D0
:1026F0000020C0462005E90A0843009908436905FF
:10270000F20A114358E60000FF070000FFFFFF7FB9
:1027100010B5002801D002F08BFF10BD10B50146A6
:1027200002A000F03DF8012010BD000053494752BF
:10273000545245443A2052656469726563743A2084
:1027400063616E2774206F70656E3A200000000090
:1027500010B5012805D0002103A000F021F80120C8
:1027600010BD09A1F8E7000053494752544D454DAB
:102770003A204F7574206F662068656170206D6522
:102780006D6F7279000000003A2048656170206D1D
:10279000656D6F727920636F727275707465640015
:1027A00070B505460C460A2000E06D1C02F0C0FF23
:1027B000002D06D028780028F7D102E0641C02F032
:1027C000B7FF002C02D020780028F7D10A2002F0B1
:1027D000AFFF70BD70B58C180578401C6B075B0FA0
:1027E00001D10378401C2A1106D10278401C03E075
:1027F0000678401C0E70491C5B1EF9D12B0705D4CE
:102800000023521E0DD40B70491CFAE70378401CBC
:10281000CB1A921C03E01D780D70491C5B1C521EE4
:10282000F9D5A142D8D3002070BD00000549064A61
:102830008A42104600D105488A4200D10449FDF77A
:102840006CBDC04600800130F07A0030E87A00307C
:102850000020003080B503F037FE80BC01BC864606
:1028600003F0C4BCB0B560B1044600F03DF90546C4
:10287000204600F091F8284381B2042001B90846AF
:10288000B0BD0220B0BD000020B11149096809B1F6
:10289000096A08470220704721B10D4A12680AB13F
:1028A000526A1047022070470949096809B109684E
:1028B000084702207047C04622B1054B1B680BB188
:1028C0009B69184702207047014908600020704743
:1028D000DC790030B0B543684C680122A3420FD1C7
:1028E000002253B189688068002204780D78654021
:1028F0002A43401C491C5B1EF7D150421043C20FB3
:102900001046B0BDF0B503AF83B06E46002202247E
:10291000204BC1B331600023DA43022400287360E6
:1029200008D14B4800684B49B1FBF0F14A1C4243C7
:1029300000231C4648480068C11D0725A9436D4671
:10294000B5606D466D1AAD4682B06946086028468E
:1029500002F00EFF02B00028B068726810D128465D
:10296000316803F015F80446020C0A48044206D107
:102970003B48016819B10720154688472A46B068C8
:10298000854604490B461C4010040019FC1F053CF9
:10299000A546F0BDFFFF0000F0B581B00224D0B124
:1029A000054602F0DFFE064602F0D4FE2B4F3860EB
:1029B00002F0C8FE26490860386840F22711B1FBD2
:1029C000F0F1491C41432448016026B924480560C0
:1029D00000242046A847204601B0F0BDF0B583B0E2
:1029E00002248AB30346906870B30026F54302249C
:1029F0003BB9174B1B68174CB4FBF3F4651C5D43E4
:102A000000245768144B1B686FB1144E029119468D
:102A100033687E1EB6FBF3F6761C5E430B460299C6
:102A20001268964210D86A4616606918CA180025BE
:102A30002B4602F09DFE38B90948016800292C4652
:102A400002D0042088470024204603B0F0BDC046D1
:102A5000EC790030FFFFFF03E4790030E8790030C3
:102A6000E0790030F0B5A1B004460026022014B38E
:102A700000261F961E961EA8194D0822294602F010
:102A80007FFFB8B91EAF384603F00BF80190381D30
:102A900003F007F802280DD102A87021FEF743F9D0
:102AA00010480199814205D102A87022294602F0FE
:102AB00067FF28B1042080B23104081821B0F0BDAE
:102AC00002A8214602F0BEFF060C0104F3D10E4815
:102AD000016800200029EED0062088470020EAE7A0
:102AE00000200210D4B3515AB0B5044602F004FFDE
:102AF000022530B904480460002514B10025284699
:102B0000A0472846B0BDC04608390030F0B5BFB078
:102B1000584C002800D18AE08768002F00D186E059
:102B20000E46002900D182E04568402D00D97EE0A4
:102B3000002A00D17BE0B068002800D177E09068DF
:102B4000002874D01068202871D301922FA840214A
:102B5000039136220292FEF7BFF81FA85C22039968
:102B60000392FEF7B9F8FDB13878029948402FA9D1
:102B700008703878039948401FA90870012D13D0B8
:102B8000681E1FA9491C7A1C2FAB5B1C1D78177887
:102B90006F400D781F7017786F400F70401E491CF2
:102BA000521C5B1C0028F1D104AF384603F02EFE06
:102BB0000021384603F05EFE68BB04A82FA940221E
:102BC00003F0A8FE38BB7268B16804A803F0A2FE47
:102BD00008BB0198816804A803F084FDD8B904A853
:102BE000002103F047FEB0B904A81FA9402203F05A
:102BF00091FE80B90198816804A82026324603F02E
:102C000089FE40B90198816804A803F06BFD10B9F2
:102C100001984660002404A803F0F3FD2FA8402586
:102C2000294603F053FD1FA8294603F04FFD204617
:102C30003FB0F0BD70B584B0044601680D4D202949
:102C400011D3A06803F03EFB68B90B4801A90A46FE
:102C500068C868C21020606020462246FFF756FF11
:102C60000546002025B12168A068FEF75AF82846DD
:102C700004B070BD01004355147A0110FEE7F0B5B1
:102C800000231C460125A5400D4207D015469D4056
:102C900003269E400768B7432F4307609B1C641CB4
:102CA000102CEFD1F0BDF0B500231C460125A54046
:102CB0000D4207D015469D4003269E40076BB74343
:102CC0002F4307639B1C641C102CEFD1F0BD00F058
:102CD00049FEFDF781FAFEE710B514494218415844
:102CE0004C0001218B07002C06D511494058C00328
:102CF00017D5F648002116E012681A4214D140F6A2
:102D000020028158802319438150094941580124E8
:102D100024040C40210CED4C217284589C438450B7
:102D200002E0EA4801210172084610BD28080000AF
:102D30002C080000F0B585B00446E44E7268092105
:102D400001AB00F045FB3068C11E324F01980129EC
:102D50002AD8800F032836D3726807210025204621
:102D60002B4600F0DBFA40F208402B4921502B485B
:102D70002750082120462A4600F064FB002847D14E
:102D8000254D07210022204600F08CFB40F6200054
:102D9000215840220A432250201801684906FCD4D9
:102DA000D420285841082FE0800F039902981CD0A6
:102DB000090C8006800A40184002C019401C4100DE
:102DC000F160306122E003988103490F04228A40B8
:102DD000800F02998B051B0D1818401C50430903E6
:102DE000090F8840810A400A0EE08A03520F04232B
:102DF0009340890F8205120D5118491C5943000355
:102E0000000F8140480A890AF0603161781C7061C6
:102E100005B0F0BDFF01000050340030380800005C
:102E2000F0B589B0044640F2001640F200112C3192
:102E300000F024FC40F62000215820220A432250B2
:102E40002018C64F397A0268920603D50029FAD1B4
:102E5000C148E0E0002120460A4600F023FB41F291
:102E6000000001E00898401E089008980028F9D159
:102E700075480125057075480290029B40F20012CA
:102E800055320821204600F049FA08900898002899
:102E9000019535D0002120460A4600F003FB089634
:102EA00002E00898401E089008980028F9D1029B7B
:102EB0003721002520462A4600F030FA089008986D
:102EC00002284ED10025204629462A4600F0EAFA7B
:102ED000089602E00898401E089008980028F9D14A
:102EE0005B4E01273770029B5B4A2046394600F053
:102EF00015FA02283BD1994805609748401C8AE0A2
:102F0000029B37210022204600F008FA5048057045
:102F1000029B29212E46504D20462A4600F0FEF9FC
:102F200040F63000271820580102F605002911D478
:102F3000029B37210022204600F0F0F9012044498D
:102F40000870029B292120462A4600F0E7F93868DC
:102F50003042EDD002224002019D00D52A46E94FC1
:102F600031E00898D8B13D60E548401D53E040F697
:102F70003000251820580102FF05002909D401213D
:102F80003170029B2046344A00F0C8F92868384264
:102F9000F5D003220421400213D50A4611E02C4843
:102FA000019D0570029B29212A4A204600F0B6F9AE
:102FB00040F63000271820580002EE0502220028B3
:102FC0002BD5D04F019D3A600221002203AB204651
:102FD00000F0FEF93868C01E01280AD82D0403212C
:102FE000002320462A4600F099F9079048B97D60F1
:102FF00010E0032100222046134600F08FF90790CD
:1030000008B1079807E040F6300020580002134945
:1030100001407960002009B0F0BD0092019D029B43
:1030200037210022204600F079F9E8480570029B1C
:1030300029212046074A00F071F938683042EED065
:10304000DF4F009ABFE7C04648340030FFFF0F0053
:103050009C7900300080FF000080FF400000FFFFEF
:10306000F0B581B00091044640F20040022727509D
:10307000201840F60001661801688907FCD4012574
:103080000560032030603068C007FCD1EC4818218F
:10309000FDF749FE37600E482158AB070A461A4330
:1030A0009943009B9B0500D50A462250215840F2C7
:1030B00000120A432250316A44F200000143316297
:1030C000316A0142FCD101B0F0BDC0462C34003061
:1030D00028080000B0B504461E480021215040F6E3
:1030E000200021580F221206914321502158092215
:1030F00012060A4322502158FF2212049143215004
:10310000215801252A040A432250215848F200027E
:10311000914321502046FFF7DFFD48B12046FFF7DD
:103120007FFE88B9F0480068032803D10D4902E00A
:10313000EE48B0BD0A4900F0A1FA2046FFF7FAFDBB
:10314000204600F0D5F900B1B0BD07480560002069
:10315000B0BDC046040800001001FFFF2C34003051
:10316000A8610000204E000044340030F0B589B062
:103170000024089440F6200404900719DB48C41C7E
:103180000393002B00D18DE002920E46D648426890
:1031900007210025049C20462B4600F0BFF805902F
:1031A00008B1059C7EE00195029B386840252843C4
:1031B000386038684006FCD4F8680006F5D55248F7
:1031C00052492150C8480068012802D0042800D084
:1031D0005B02C348235040F208402650FF20039969
:1031E000B1FBF0F102910691069A82B3BE4A127ABF
:1031F0004749484E019B33703C680C4007940404D7
:10320000079B23430793089B079C1BB104231C4384
:103210003C6004E040490C433C6001230893337850
:1032200023B9337813B9002AF9D13AE0AF4B9C1D8A
:10323000FB685B0736D5AD4BDC1DFB681B0731D542
:10324000069B5B1E0693069B002B3149D2D1029947
:103250004143039A511A0691069981B32D49019A67
:103260000A703A6843F600739A4307920004079A7B
:103270008243079206980004079A02430792089A2D
:1032800007981AB104221043386004E0224A104320
:103290003860012008909448007A0A782AB90028FA
:1032A000FBD1924C204609B0F0BD9048841DF868CF
:1032B0004007F7D58D48C41DF8680007F2D50C21EA
:1032C00000220498134600F029F888498C1D002834
:1032D000E8D138682843386038684006FCD4F8687C
:1032E0000006F6D5072100240498224600F0DAF8FB
:1032F00038682843386038684006FCD4D2E7C046B6
:103300001001FFFF2C34003038080000FF010000DE
:10331000FFC0FFFF9D79003007120000B0B5704C70
:10332000025140F620028458244D254009022943C9
:10333000C91C81508118CE4A127A43B1DB430C6814
:10334000A4070BD55B1C22D0002AF8D104E00B683F
:103350009B0703D5002AFAD164492DE019490A7860
:10336000012A0BD1184A8258D2B2552A06D040F60B
:10337000300282580F231340012B19D1134A1178C0
:1033800061B100211170464A0223835014E008689D
:1033900044F2000202430A6002210DE04049405815
:1033A00042075248801D0021002A00D50846B0BDC2
:1033B000002008704D4909310846B0BDFCC0FFFF30
:1033C0002C34003048340030340800009C79003040
:1033D00070B585B0424C025140F620028458174D1A
:1033E000254009022943113181508118A04A127ADF
:1033F0000C68E40603D5002AFAD13C491BE02849B1
:1034000041584A073949891D002A14D500214258DC
:103410006C466250091D1429F9D16846001D00212F
:10342000009C0A4685582E0E240234199C50121D09
:10343000102A2C46F6D1084605B070BDEEC0FFFF3D
:103440002C34003010B5264BC25040F62002835871
:10345000124C1C4009022143C91D81508118844A25
:10346000127A0B689B0702D5002AFAD104E00B6898
:103470005B0703D5002AFAD11C4810BD084A811801
:1034800080584307194A901D002BF6D5D01D0A68B5
:103490000021120700D5084610BDC046F8C0FFFF46
:1034A0002C08000010B581B0002300930C4BC250D3
:1034B00040F6200283580B4C1C4009022143491C52
:1034C000815081188058C00707D06948007A074AA0
:1034D00000B900920B68DB07FAD1009801B010BD6B
:1034E00024080000FEC0FFFF2C3400301001FFFF55
:1034F000F0B581B004465E4842680023009307257A
:1035000020462946FFF70AFF009040F62001661882
:1035100010B1009801B0F0BD3068402738433060EA
:1035200030684006FCD4F0680006F5D5F84800681D
:10353000401E03287DD8810001A251188F46C04645
:1035400000F006B800F02CB800F056B800F059B8FA
:1035500040F208408C492150EE482550EC48426822
:10356000372100232046FFF7D9FE00900028D0D154
:10357000854D332100222046FFF764FF009000288C
:10358000C7D128780F2101400F2921D1204600F012
:10359000BBF800900098D8B95A4900F06FF817E0CE
:1035A00040F2084078492150DA482550D84842680E
:1035B000372100232046FFF7B1FE00900028A8D154
:1035C000332100222046FFF73DFF00900028A0D1C4
:1035D000CF484268372100232046FFF79FFE009026
:1035E000002896D10621022200232046FFF796FEEE
:1035F000009000288DD117E0306848F20001884320
:10360000306006211B4A00232046FFF787FE00900A
:10361000002800D07DE730683843306030684006CD
:10362000FCD4F0680006F6D5306848F2000101438A
:103630003160B94D6A1C102100232046FFF76EFE51
:103640000090002800D064E7B248255007210022EE
:103650002046FFF727FF3068384330603068400667
:10366000FCD40548215801220A432250002051E78A
:103670002C3400300001B70328080000B0B50C4618
:1036800001F07EFFC00038D40F20C0431B4D2858E6
:103690008002800F012805D0022806D0032807D118
:1036A00017480BE004F024F804E004F027F801E0E8
:1036B00004F02AF840F2E831B0FBF1F011498C42F5
:1036C00000D30C46B0FBF4F25443001B511C00B96C
:1036D000114640F20012FF2903D8002000290A46B3
:1036E00003D0FF20000611060818FF2109062A68EA
:1036F0008A432A60296801432960B0BD2002004046
:10370000E02E000050C30000F0B581B00446002652
:10371000009640F208411C4860507E4D3F2767519B
:1037200006211A4A2046FFF78DFE0090611940F2EB
:103730000842A218012510B1284601B0F0BD124B75
:10374000188840BA0028F7D0988B40BA0028F3D1E7
:1037500013600F6006210E4A20461F46FFF772FED7
:1037600000900028E8D13B4640F620002158402236
:103770000A432250201801684906FCD4188840BA30
:10378000351A4541D8E7C0465034003001FFFF00EC
:1037900001FFFF80F0B589B016460022089240F67E
:1037A00020028418594AD71C002B00D180E00391D5
:1037B000049357494A680721002705463B46FFF70F
:1037C000ADFD059008B1059F72E002972A46049B63
:1037D000206840252843206020684006FCD4E0682B
:1037E0000006F5D54B484C4911504948006801285E
:1037F00002D0042800D076024848165040F2084013
:10380000019203991150FF20B3FBF0F1039106914F
:10381000069A42B33E490A7A414F424E02993170AC
:10382000236839463B4007930304079F1F430797CC
:10383000089F079B1FB108273B43236004E03A4FD2
:103840003B432360012308930F46337813B9002AC2
:10385000FBD12CE0E3689B0753D4069B5B1E0693C9
:10386000069B002BDAD1039948430499081A069065
:1038700006980028029921D02A48017006992268EA
:10388000274B1340090419430791089A07991AB165
:1038900008221143216004E0234A114321600121E1
:1038A00008911B49097A02782AB90029FBD1174FE0
:1038B000384609B0F0BDE068800722D40220E060FD
:1038C0000C210022019E30461346FFF727FD0F49C9
:1038D0008F1D0028ECD12068284320602068400616
:1038E000FCD4E0680006F6D50721002730463A46AA
:1038F000FFF7D8FD20682843206020684006FCD4EC
:10390000D6E70220E060014F0837D1E71001FFFF42
:103910002C34003038080000FF01000024080000AB
:1039200080C000FF9D7900300B19000080B503F0C6
:10393000DFFE0749086003F0EDFE0649086006490E
:1039400040180649B0FBF1F00549086080BDC0464B
:103950001C3200302032003020A1070040420F000E
:1039600018320030014802490160704708ED00E05C
:103970000000011010B5044600201B498C4209DCF0
:103980001D498C4213D01D498C4212D01C498C42D7
:103990000BD021E015498C4205D015498C4204D04A
:1039A00014498C4218D1174804E0174802E00D482A
:1039B00000E0164803F0B4FE02280AD140F20010DD
:1039C00004430E48844208D110BC01BC864603F073
:1039D000ADBE80000EA1085810BD10BC01BC8646CB
:1039E00003F0AABE0200805EFF10054000110540F2
:1039F0000010055000110550000005400001054071
:103A0000001005400500405F0400005F0300C05E39
:103A1000001BB70000800000000000000000000054
:103A2000000000001027000000000000001BB7008D
:103A3000F0B585B0009104466C4801A96CC86CC112
:103A40006B4F6C4884420ADC7248844215DC75482E
:103A500084422AD07448844222D0744809E06648DF
:103A6000844212DC684884421FD06848844217D0E0
:103A70006748844221D1714F17E06748844211D0D2
:103A80006648844210D0664806E05C48844209D00B
:103A90005B48844208D05B4884420ED1644F04E006
:103AA000674F02E0644F00E0624F384603F038FE93
:103AB0000646384603F046FE471C002020630325D7
:103AC000E560A06810490140A160012E02D103F019
:103AD0000FFE0290009BABB1B00001A90858B0FBEB
:103AE000F7F158080818B0FBF3F0801E020C06D05E
:103AF000D8000818B0FBF3F00009801E01E0290788
:103B00000843606205B0F0BD0FFFF0FFF0B587B06D
:103B10001C46029201910546344803A9CCC8CCC189
:103B2000334E344885420ADC3A48854215DC3D482C
:103B300085422AD03C48854222D03C4809E02E48A4
:103B4000854212DC304885421FD03048854217D06C
:103B50002F48854223D1394E17E02F48854211D096
:103B60002E48854210D02E4806E02448854209D0D0
:103B70002348854208D02348854210D12C4E04E0CA
:103B80002F4E02E02C4E00E02A4E304603F0C8FDD6
:103B90000746304603F0D6FD0646012F03D103F059
:103BA000A7FD049001270C98019BC3B1B90003AA9B
:103BB0005158721CB1FBF2F259085118B1FBF3F1E4
:103BC000891E1E460B0C06D0F1005118B1FBF6F110
:103BD0000909891E02E00322120711436962029952
:103BE0000C430443EC6007B0F0BDC04648860110AA
:103BF000103D8057FFFF0650FF2F07500030075041
:103C000000400750005007500000075000100750B8
:103C100000200750FF2F07400030074000400740BA
:103C200000500740000007400010074000200740F8
:103C3000953DEC77143DCC77933CAC77123C8C7778
:103C4000913DA05780B501F0F9F80149086080BDA9
:103C5000F838003080B501F04FFE0021091A4841C4
:103C600080BD01F03DBE0000F0B581B004461C4EA1
:103C70003746384601F03CFEC7193046703087425F
:103C8000F7D3184DAF4209D217A001F05FFF2548C6
:103C90003918304601F0FCFDD8B903E040F200408D
:103CA000241835462F19AF4209D92E46304601F067
:103CB0001FFE8619BE42F9D31B48864204D8284607
:103CC000214601F0E5FD04E0184801F03FFF002027
:103CD000C0430021091A4141084601B0F0BDC04669
:103CE00000200210002402105B444247205D204562
:103CF000726173696E6720686561646572207365BF
:103D00007061726174656C792066726F6D20616399
:103D100074697665206170706C69636174696F6E37
:103D20000D0A000000E0FDEF00000810998A011064
:103D3000F0B589B005900020002963D00C4601F051
:103D4000D3FD314AB2FBF0F14143511A04D02F4860
:103D500001F0FCFE30BFFDE7002107912C490891DE
:103D600044F20001B1FBF0F1049041430691A368D5
:103D7000E2681D461543083402940120002D41D00D
:103D80000498401E01900020224E074603901BE03D
:103D9000079898B31C497918019A1018049AB0FB37
:103DA000F2F5554308982A4601F0AAFD0146002481
:103DB000201A4841EF19029A13685268FD1A94417B
:103DC00020D2F9B900200699039CE5433560DB1B3E
:103DD0008241C81A2046904100D31946079106AA8D
:103DE00005983946FEF768FD0004306802D003E00C
:103DF00030BF3068411CFBD00428C9D006A001F0B8
:103E0000A5FE002009B0F0BD00240210898A01102F
:103E100010390030643200305B444247205D20415D
:103E2000524D5F5543505F526561642072657475F1
:103E3000726E656420302062797465730D0A00002B
:103E400070B50C46064611A001F080FEA068FFF791
:103E50000BFF0025B8B116A001F078FE204600F057
:103E60004DF980B118A001F071FE30462146FFF7F0
:103E70005FFF40B11BA001F069FE204600F040F852
:103E800000210D1A4541284670BDC0465B4442479B
:103E9000205D2045726173652061637469766520D9
:103EA0006170706C69636174696F6E0D0A00000067
:103EB0005B444247205D20577269746520686561E4
:103EC0006465720D0A0000005B444247205D204398
:103ED0006F7079206170706C69636174696F6E0DC9
:103EE0000A0000005B444247205D20566572696607
:103EF00079206170706C69636174696F6E0D0A007E
:103F0000F0B5A7B00125002854D0044600F0DCF835
:103F100000284FD0A068E1680143274608370225F2
:103F2000002947D002940CAE304602F06FFC00210D
:103F30003046019102F070FC04A82021FCF7F3FE4A
:103F400003973868E0B1984E074602E0C7B103987E
:103F5000006844F200018F423C4601D344F2000461
:103F60001649C91B09183046224601F009FD0546CD
:103F70000CA83146224602F0CBFC3F1B002DE5D0B9
:103F80000CAD04AE2846314602F0AAFB284602F0EA
:103F900038FC029C1034202220463146FCF7F4FD08
:103FA0000028019D06D0204602F004FF04A802F07C
:103FB00001FF0125284627B0F0BDC04600240210AD
:103FC000F0B5A1B002900020002962D00D46324821
:103FD0001EA91CC81CC103AE304602F017FC00210C
:103FE000304602F019FCA968E8680A4602430095C9
:103FF000083501959AB3002444F20002274D264665
:10400000234610E01F9A3AB3209903A802F080FCDF
:104010001F9886190198016840680022731A82412E
:104020001DD200231E9AE7432F60891B9841531A23
:104030002346834100D30A461F921EAA02983146A6
:10404000FEF73AFC0004286802D003E030BF28687D
:10405000411CFBD00428D5D011A001F077FD03ADA1
:10406000514E2846314602F03BFB284602F0C9FB80
:10407000009C1034202220463146FCF785FD014685
:10408000012031B1204602F095FE474802F092FE31
:10409000002021B0F0BDC046207A0110643200300B
:1040A0005B444247205D2041524D5F5543505F5273
:1040B0006561642072657475726E6564203020627B
:1040C000797465730D0A0000B0B5002488B100242E
:1040D000E143094D2960FEF7D7FB000409D100E058
:1040E00030BF2868411CFBD0062801D1012400E024
:1040F00000242046B0BDC04664320030F0B587B021
:104100000025E943002843D003900191029501F076
:10411000EBFB07466F37B7FBF0F141437E1A1E4CAD
:104120002546284601F0E4FB4519204670308542BB
:10413000F7D3BF1B1948874208D21A48281887426C
:1041400009D9174801F002FD30BFFDE7144801F01E
:10415000FDFC30BFFDE71448FF223946FCF7B3FDF4
:10416000124804A90A4668C868C2039801F02EFBE9
:10417000000402D0029D01990AE005987028029D72
:10418000019905D1084821463A4601F0B9FB01469C
:10419000681A484107B0F0BD00200210014000003D
:1041A000898A011000E0FDEF103900302C7A0110EF
:1041B000F0B595B0039300250B950A9509950895E0
:1041C0000795069505950495424C002A7CD00F462C
:1041D0000646029208A800F0A7FF0E34002873D10B
:1041E00008A8314601F0A4F930468F30B8420BD808
:1041F00008AC204601F09AF90190204601F092F9AE
:1042000001994018B84201D2324C5AE0B81B441C04
:104210006708314608D00025314608A801F088F922
:104220004519A919BD42F8D31A9801900496069130
:104230000595601B0790002508AC204601F074F935
:104240000746E80004A90E58324640320CA908235C
:10425000204600F081FF78BB00200CA9095C401CBF
:10426000B94202D10728F8D926E00CA8478801985E
:1042700000B10760039887421ED808A80299324609
:104280003B4600F069FFB8B90EA801218181017594
:104290000023D9430F91104908310E9110930F4913
:1042A000129114A96A46116002993A4600F060FE24
:1042B00014980D9988420AD06D1C022DBCD3054874
:1042C000841D08A800F05EFF204615B0F0BD002454
:1042D000F7E7C0460101FF800486011050810110FC
:1042E000F0B5ABB018A848242146FCF71CFD06AD7C
:1042F00028462146FCF717FD2846FFF701FE5B49DB
:104300000B6800249BB158490A6882B1C0CB079C56
:104310006740069D6E403E43083B16B913785B1C10
:1043200002E01D605C600023137009680C780126B0
:1043300002280CD068B9022C0DD806A8103002F063
:1043400039FD0798199006981890344609E048A05E
:1043500004E0032C01D35CA000E04FA001F0F6FBC9
:1043600000240020C143634D2960049405967440E5
:1043700006AE3146FEF790FA01043246303218AFED
:104380003B46303338461030029008373046103004
:1043900003900836286811B103E030BF2868411C3B
:1043A000FBD0072847D10093019230480568079851
:1043B0000699002D059A07D02B686A6842404B4049
:1043C0001343012203B91A46199B189D691A8341A8
:1043D00033D22243012A30D103CE0143083E61B3D8
:1043E000002406A92046FFF7EBFDB8B3039D28463D
:1043F00002F0E0FC03CE434A821A0A46A2412FD2C1
:10440000079A1992069A189203C7029C0FCD0FC4FF
:104410000FCD0FC4019C009D0FCC0FC53D4801F08E
:1044200095FB002018A9FFF70BFDD8B13B4801F020
:104430008DFB059C0FE0304800E0304801F086FB22
:10444000059C049818B1324801F080FB03E02F4826
:1044500001F07CFB002420462BB0F0BD2848EDE79E
:104460002948EBE72C48F3E70C390030A0790030FD
:104470005B444247205D204163746976652066692C
:10448000726D7761726520736C6F7420697320653B
:104490006D7074790D0A00005B444247205D204135
:1044A0006374697665206669726D776172652069EB
:1044B0006E7465677269747920636865636B2066E2
:1044C00061696C65640D0A005B444247205D2046CB
:1044D00061696C656420746F20626F6F7420616322
:1044E00074697665206170706C69636174696F6E60
:1044F0000D0A000064320030938B0110028C011011
:10450000268B011001DC0500A58B0110728B0110B8
:10451000DE8B0110BE8B0110068B01104C8B01103D
:10452000F0B589B00F460646002508950795069513
:1045300005952748306027480860274CE01C316803
:10454000002943D005A800F0EFFD014620460930C0
:10455000E1BB049705AF2149384600F0E9FF384632
:1045600000F0E4FF0390384600F0DCFF029034686E
:104570003846214600F0DCFFB4FBF0F444430498D5
:1045800000680190411E384600F0D2FF07463068AF
:10459000A04217D10198401E2946A9413A462B4610
:1045A000FBF794FF401C78430399029A5218049930
:1045B0000968914206D8814204D105A800F0E2FDC5
:1045C000002003E005A800F0DDFD034809B0F0BDC0
:1045D00000000210002002100601FF80D08E0110A2
:1045E000B0B50E4800F012FE0D480C300021CC434F
:1045F0000325016859B1001D6D1C102DF9D3FBF77F
:10460000D1FE18210160054800F000FE04E00460BE
:10461000024800F0FBFD2C462046B0BD5836003065
:104620002432003082B080B582B00593049220B16C
:1046300004AA01920348FBF7CAFF02B080BC01BC88
:1046400002B00047C03300302649096801B108476D
:104650007047C046364800680168084734484068DB
:104660000168084732488068016808473048C068D8
:10467000016808472E480069016808472C484069CE
:10468000016808472A488069016808472848C069C6
:104690000168084710B582B0044601F0A1FA002174
:1046A0002448234A136873B1121D001D491C0829B0
:1046B000F8D301F0D7FA002268460260074808499B
:1046C000134601F087FE1460046801F0CBFA054838
:1046D00005490160204602B010BDC046200101809E
:1046E0002287011080380030ED46011010B582B0ED
:1046F000044601F075FA00210D480E4A1368A342E2
:104700000ED0121D001D491C0829F7D301F0AAFA8A
:10471000002268460260084808A1134601F05AFECC
:104720000021016002B010BC01BC864601F09ABABB
:1047300060380030308101100101018054726965D8
:104740006420746F206672656520696E76616C699D
:104750006420435468756E6B456E74727900000076
:1047600010B500202AB10C461C4802F031FC207024
:10477000012010BD1C20C04370471520C043704766
:1047800000207047F0B581B014464AB10D46134E73
:1047900027462978304602F0E9FC6D1C7F1EF8D1CF
:1047A000204601B0F0BDC0460120704770B50446F8
:1047B0000848083020600848006840B91546074E90
:1047C000304602F0CFFC3046294602F08BFB2046F3
:1047D00070BDC04650850110DC7A0030F47900309D
:1047E000FBF715BEF0B581B004464C20205C264690
:1047F0004C3620B1206D401C206500255EE0002075
:104800002065204600F0D0F90546002856D1E06822
:10481000002856D014214556E06A08B1E9B206E0F6
:1048200020461830FFF736FFE062E168097DAA00F4
:10483000264B1B689A18106448B2002808DBC10890
:10484000032291431F22024001209040204A8850B9
:10485000606940F20011FEF703FC6069FEF73AFC64
:104860000F200705A07C0006000F01D032780CE075
:104870001848016801220029104600D1084616494F
:10488000096801B90A46024032701AB10120206558
:10489000002505E0207A11A1FFF7C4FE3278164DFD
:1048A000207A16A1FFF7BEFE2069384201D0606869
:1048B00002E00848C0686060211D0860284601B019
:1048C000F0BD12481249DA2201F0F0FC08ED00E0D8
:1048D00000E100E02C340030443400304661696C63
:1048E00020746F20696E697469616C697A652063F0
:1048F0006172640A000000005FF0FFFF696E697476
:104900002063617264203D2025640A005C860110EA
:1049100071860110F0B587B01D46174606910168F3
:10492000C96B0D9C6A4654600C9E166003903A4613
:10493000884701467E4A501C00295ED04C200399CE
:10494000085C0028104658D0049705950321069D61
:104950002A460A40774B3046184010430F22120770
:104960002A4001239B075B1BB34212D309078A42EB
:104970000FD170B90498400A0599C9054218700A08
:10498000E1054318039840690699FEF7EFFB98BBD1
:1049900033E03146214300200029059A049B2CD0A6
:1049A0000493580A0592D1054218700AE10540188F
:1049B0000294610A01435F48451C01B935466B0A00
:1049C000039840695C4C2146FEF7D0FBA0B9069FD6
:1049D000384621462A46FCF727F90020761B029C20
:1049E000844131462143049B5B19059A42417F195A
:1049F00006970029D4D100E0D44807B0F0BDC046E6
:104A0000017270474C21415C002001B94848704751
:104A1000B0B504464C20215C25464C35002059B1E8
:104A2000206D022801D3401E06E0E06810B1406806
:104A300002F08EFE0020287020650020B0BD00002E
:104A4000F0B587B01F4614460D460168096C0D9EEF
:104A50006A4656600C9B06931360059022463B46BF
:104A600088470146324A501C00295ED04C200599E7
:104A7000085C0028104658D00394049703272A4660
:104A80003A402C4B06990846184010430F22120753
:104A90002A4001239B072C465B1B0D468B4212D3F9
:104AA0003B079A420FD170B90398400A049AD20585
:104AB0008218680AF305C318059840692146FEF775
:104AC00069FE88BB31E02A46334632430020002A83
:104AD0002746049C039E28D02946480ADA058018F8
:104AE00004935A0A02431348451C02B90D46069125
:104AF000114839462A46FCF797F8700AE105421832
:104B00006B0A059840690C49FEF744FE60B9002025
:104B10000699491B049B83410A461A43761944416E
:104B20007F19002AD9D100E0884807B0F0BDC046FF
:104B300074ECFFFFFF010000603600304169174A46
:104B400088188A58D20706D00122026040F6000079
:104B50000B5813430B50124A88188958C90703D0C1
:104B6000104901220A7002600168C90502D540F2AD
:104B7000001101600168890701D502210160016807
:104B8000890402D542F2000101600168C90404D51C
:104B900041F2000102680A43026070470808000001
:104BA0002C0800009D790030F0B581B00446007AF1
:104BB00049A1FFF737FD206B514901F0B1FF00908B
:104BC000606B504901F0ACFF0646A06B4E4901F006
:104BD000A7FF0746E06B4D4901F0A2FF054600988C
:104BE000314601F07DFF06463846294601F078FF40
:104BF0000146304601F074FF0090206C444901F0FA
:104C00008FFF0646606C434901F08AFF0746A06C9F
:104C1000414901F085FF05463046394601F060FF05
:104C2000294601F05DFF0146009801F059FF054655
:104C3000401C3CD03949284601F032F8E060F0B31E
:104C40000068A84241D1206B2D4901F09BFF606BA9
:104C50002C4901F097FFA06B2B4901F093FFE06B0B
:104C60002A4901F08FFF206C294901F08BFF606C0D
:104C7000284901F087FFA06C274901F083FF3148E4
:104C80002E46064002F06AFD25616661E068006913
:104C900002F06AFDE268121D07CA02F06BFDE068CF
:104CA000406802F06DFD02F071FD002005E0206813
:104CB000C26C012120469047244801B0F0BD224833
:104CC0001F4940F2D81201F0F1FA40F2D810421C0C
:104CD00013A01B4901F0EAFA5344204D50462053DB
:104CE000657474696E67202620456E61626C65206C
:104CF000534420495020436C6F636B0A000000004E
:104D0000A47B0110C87B0110EC7B0110107C01100A
:104D1000807B01105C7B0110387B0110F880011052
:104D20005F7364685F6D6F64696E69742D3E6D6F4B
:104D3000646E616D65203D3D2073645F6D6F64003E
:104D400071860110E0FF0FFF5C8601105FF0FFFF2E
:104D5000F0B5002141600172C16041610162124AF7
:104D600042628162114A8261114F204B0833036015
:104D7000CB4303613B46F5333C46F6343D46F735BD
:104D80003E46F836FA370A4AF932C1620363446391
:104D90008563C66307644264054A8264C0614C222D
:104DA00081540165F0BDC0463D4B0110B551011065
:104DB0000D03000080B500F005F880BC02BC8E46F3
:104DC00000F0BABB10B504460848083020604C20FB
:104DD000205C10B12046FFF71BFEE06A18B1FFF718
:104DE00033FC0020E062204610BDC046AC850110B7
:104DF0001520C04370471820C243002001B9104657
:104E000070471520C04370470168896A0847002031
:104E1000704701680B690021012218470168896900
:104E2000084703681B691847704701680B69002130
:104E30000A4618471520C0437047704710B50D4803
:104E40000078BFF35F8FC00701D00B4810BD094841
:104E500000F09AFB0028F8D0074C2046FFF778FFB7
:104E60000648074A214600F08DFB024800F0B6FBD9
:104E7000EBE7C04654360030A0380030C54D011075
:104E800000000110002070470020704770B500241A
:104E90000F281ADC0546800015490C580E18022D03
:104EA00013DC601C11D1284600F02AF8044658B9DA
:104EB000284600F027F8044630B90E480078BFF3C2
:104EC0005F8FC0070C4C02D03460204670BD09488B
:104ED00000F05AFB0028F7D0E1204202064C0749B7
:104EE0002046FFF763FC034800F078FBECE7C04680
:104EF00024320030503600309C38003018860110C3
:104F0000002070470020704790B4047D022C04D02C
:104F1000012C05D190BC00F079BA90BC00F0B6BA73
:104F20000020C04390BC704770B5C1B10A68437B94
:104F300063B100232024D50703D0651E0126AE40AF
:104F40003343641E5208002CF5D100E013468268FA
:104F50005A400A60016889688847002070BD164879
:104F6000164940F2131201F0A1F9C0467047000043
:104F700070B582B0069CD4B1054640682060684692
:104F800004602846FFF7C0FF28B1064628688168FC
:104F90002846884708E028462146FFF7C5FF002637
:104FA00010B1002121600646304602B070BD0248B3
:104FB0000249A12201F07AF9A6860110B2860110F9
:104FC00000F0BABA7047007B70470000F0B581B0BE
:104FD0000E460446174800F019F9174805680DE019
:104FE000AF6857B13846FBF7FDFDB04205D13846F2
:104FF00021463246FBF7C8FD88B16D68002DEFD120
:10500000072E05D10DA007222146FBF7BDFD50B1AB
:10501000084800F0FBF80025284601B0F0BD05481F
:1050200000F0F4F8F8E7034800F0F0F805480568E8
:10503000F2E7C04688380030843800306465666125
:10504000756C740090380030B0B505464068002497
:1050500038B1FFF7B8FF012803D16868041F00B911
:1050600004462046B0BDB0B505464068002430B1C6
:10507000FFF7A9FF18B96868041F00B90446204665
:10508000B0BD4168012001B90846704780B541684C
:10509000002031B10846FFF796FF01460020401A74
:1050A000484180BD0068704770B50E460446002533
:1050B000056045600EA13046FBF756FD301802E052
:1050C0002F2A06D06D1C41192160425D002AF7D1BC
:1050D00001E0491C21602DB12946FFF777FF606090
:1050E000204670BD03A006A12A2201F0DFF8C046C9
:1050F0002F0000006C656E20213D20300000000074
:105100002E5C6D6265642D6F735C706C6174666F8C
:10511000726D5C736F757263655C46696C65506136
:1051200074682E637070000070B50546204E3046DE
:1051300000F06CF8284602F02FFB0446284602F0E7
:1051400031FB00F0FBF9E860304600F05FF800202A
:10515000C04304B9204670BDF0B581B01C46154669
:105160000E460746124800F051F8384629463246A6
:10517000234600F08DFD04460D4800F047F8204618
:1051800001B0F0BDB0B50546094800F03FF828462B
:1051900002F00EFB0021CC4300B90446E86808B1D8
:1051A00000F0C8F9024800F031F82046B0BDC04612
:1051B0009438003030B4436873B1C2680569012483
:1051C0002C402146114339B18168681018180CB180
:1051D00003689A5830BC104730BC7047B0B50D46D4
:1051E0000024C80705D0084801F0D0FF012400B909
:1051F0000446E80606D5044801F0D0FF21461031E8
:1052000000B10C462046B0BDF479003080B50146AF
:10521000006808B9086818B1091D884203D180BD2B
:10522000081D086080BD02A00AA18B2201F03EF893
:1052300070203D3D207265696E7465727072657490
:105240005F636173743C54202A3E28265F64617456
:10525000612900002E2F6D6265642D6F735C706C88
:105260006174666F726D2F53696E676C65746F6ED3
:105270005074722E68000000002140F20020704738
:10528000002140F200207047002140F200207047CA
:10529000002140F2002070474C21425C0021C943AC
:1052A0001AB1406840020021704701487047C0466B
:1052B00074ECFFFF00A070474E55534400000000FF
:1052C00001207047F0B585B01D46164604460068BB
:1052D000416A2046884702460B4630462946FBF77E
:1052E000F5F8134300270BBB019603950B9D0A9E0F
:1052F0002068416A2046884702460B46029630469F
:1053000004952946FBF7E2F813437BB9029801990B
:105310004618049D039845412068816B20468847C4
:1053200001270022801BA94100D21746384605B04C
:10533000F0BDF0B581B01C46174605460068016B0C
:105340002846884702460B4638462146FBF7BEF8FA
:1053500013430026EBB907980699CF19444100265C
:105360007A1E2346B3412868016B284688470246C7
:105370000B4638462146FBF7A9F813434BB928687A
:10538000816B2846884701260022C01BA14100D21C
:105390001646304601B0F0BD0020C0437047F0B55E
:1053A00085B01D46164604460068816A2046884737
:1053B00002460B4630462946FBF788F81343002780
:1053C0000BBB019603950B9D0A9E2068816A2046BF
:1053D000884702460B460296304604952946FBF75D
:1053E00075F813437BB9029801994618049D0398F8
:1053F00045412068816B2046884701270022801B99
:10540000A94100D21746384605B0F0BDF0B587B0C7
:1054100006910C9CA4B3114619430194256851B31D
:1054200001690391007B029000273C46059304929A
:105430000698C65D029860B100210823F20703D0E8
:105440005A1E0120904001435B1E7608002BF5D1C7
:1054500000E0314600207F1C4441280EC9B2414083
:105460008800039908582D024540049AB81A20462E
:10547000059B9841DCD301980560002007B0F0BD82
:105480002648274940F2D91200F010FFF0B587B046
:1054900005910C9CD4B3114619430194256881B33E
:1054A0000392007B029000261B4F31460493069125
:1054B0000598805D029961B100210823C20703D0DD
:1054C0005A1E0124944021435B1E4008002BF5D155
:1054D00000E001460906694008204D002B467B404C
:1054E000002900DA1D46401E01062946F5D100209C
:1054F000761C069941410398301A0846049B98414E
:10550000D5D301980560002007B0F0BD03480449D9
:1055100040F2AD1200F0CAFEB71DC104A68601100C
:10552000B286011002F04AB902F04EB902F052B947
:1055300002F056B9FAF76BBFFAF769BF10B582B03F
:105540000446FAF733FF08B102B010BD00236846E5
:105550000360024802A1224600F03CFF1F010180C7
:105560004F70657261746F72206E65775B5D206F3E
:105570007574206F66206D656D6F72790D0A00007D
:10558000704670470120704780B5014603780322BA
:1055900013400020012B04D00B781A4012B1012ACD
:1055A00005D180BD022003430B70012080BD02A005
:1055B0001349094A00F07AFE286775617264202653
:1055C000204358415F47554152445F4D41534B2959
:1055D000203D3D20300000009D06000080B5017890
:1055E00003220A40022A04D1FC221140491C017006
:1055F00080BD02480249034A00F058FE7588011038
:10560000AC880110A606000090B406480168762216
:10561000054B10C910C3521EFBD10349016090BC59
:1056200000F054BF08ED00E00030003000F0B6BAE2
:10563000FEE710B5FFF72AFC092430B10168896A3A
:105640008847002800DB10BD4442FAF7ABFE046037
:105650000020C04310BD00F0A1BD0000B0B50D4654
:1056600004462249FBF762FBB8B121492046FBF70B
:105670005DFBA0B11F492046FBF758FB88B120789D
:10568000402814D16078A17809020818E1782279BD
:105690001202511809040C1807E0002402E001244A
:1056A00000E002242046FFF7F1FB2046B0BD0120B8
:1056B0000221AA0700D508466907890F03D12807E8
:1056C000C1170920084040F2002141182A07920F13
:1056D00000D00846290240F200420A4081182046C4
:1056E000B0BC04BC964601F071B9C04638860110C2
:1056F0003F86011030860110002200F060BD10B519
:105700001446002A0CDB024600203CB1104622461B
:1057100001F0D7FF0021C943002807DB211A05E06B
:10572000FAF740FE162101600020C143084610BD73
:1057300080B582B001A908700120024601F0C1FFC6
:1057400002B080BD80B5124800680168C96A884708
:1057500080BDC04680B50E4800680168896A8847E8
:1057600080BDC0460A480068016889680847C0468D
:1057700070B582B001460648006804686469002577
:105780006E467560069D3560A04702B070BDC0468C
:10579000F838003070B5002299B10022D3430A4A8C
:1057A00005785D40491E08246B081E465640ED07EB
:1057B00000D03346641E1D46F6D1401C0029EFD1AF
:1057C000DA43104670BDC0462083B8ED70B506467A
:1057D0000220BEB30C46A9B32168702932D3A06859
:1057E00070252946FBF79DFAA068174900F08EF94D
:1057F000A068001D022100F089F90CCEA0680830D5
:10580000083E00F08CF9B268F368A068103000F030
:1058100086F9A0683146103118302022FBF704FACF
:10582000A0683036583010223146FBF7FDF9A068E9
:105830006C21FFF7AFFF0146A0686C3000F066F9FD
:105840006560002070BDC046D4B3515AF0B581B038
:105850000E4605464D4F384601F0BCFF044638461B
:1058600001F0ACFF0019A84210D9AC420DD2474F4D
:105870003846214601F0B4FF0419AC42F8D3201A8F
:1058800006B92046AC4200D00446204601B0F0BD27
:10589000F0B581B00D4604460121FFF7D7FF009017
:1058A000281900273946FFF7D1FF0546FE43009827
:1058B000A04211D1A5423E460ED9344F384621466A
:1058C00001F094FF06463846214601F089FF04198D
:1058D000AC4201D2002EF1D0304601B0F0BDC0463E
:1058E0002A4801F065BFC046284801F05BBFC046AA
:1058F0000146264801F074BF244801F04DBFC04660
:10590000F0B583B00025EF43019010B300921F4E15
:105910003046029101F05EFF0446304601F04EFF32
:10592000029A944215D80119009EB218B04210D3C1
:105930008A420ED8154801F035FF02990346B1FBA3
:10594000F0F05843081A04D1B6FBF3F05843301A6C
:1059500002D0384603B0F0BD002E2F46F9D0002407
:1059600009190198021909481D4601F045FF07462B
:1059700064190028EDD12B46B4420299F0D3E8E730
:1059800013460246014800F083B9C046FC38003097
:10599000F0B599B0022600284ED00C4600294BD015
:1059A000054611AE202730463946FBF7BCF90020EA
:1059B0000F900E9710960EA8FDF73CF902260004F2
:1059C0003AD1E8200C900B900D9503AE3046394645
:1059D000FBF7A9F90197009702960EA80BA96A4652
:1059E000FDF794F802261649084225D10C970B972B
:1059F0002846E8300D900BA86946FCF76BFFD8B934
:105A00002846083000F05BF803C428461030083CF4
:105A100000F055F8A060E1602046103029461831AA
:105A20002022FBF701F920463030A035102229460C
:105A3000FBF7FAF800262664304619B0F0BDC046E0
:105A4000FFFF0000F0B581B0022638B30D4629B340
:105A500004466C21FFF79EFE074620466C3000F09E
:105A600020F8B8421AD12046083000F028F803C5C3
:105A700020461030083D00F022F8A860E960284672
:105A80001030214618312022FBF7CEF8303558343B
:105A9000102228462146FBF7C7F80026304601B001
:105AA000F0BD002148B14178027812025118090274
:105AB000827889180902C0780918084670470022C0
:105AC00008B34178027812025118090282788918C5
:105AD0000902C27889180A0CFF239A430902037944
:105AE000C9180B0ED218120209024379C9180B0EFD
:105AF000D218120209028379CB18190E51181A0212
:105B0000C079121800E011461046704730B1C170DC
:105B10000A0A82700A0C4270090E0170704768B15F
:105B2000C271110A8171110C4171110E0171C370A2
:105B3000190A8170190C4170190E0170704700002C
:105B4000014908607047C04664320030B0B5044671
:105B50001048017879B90121017040F20C10411C04
:105B60000D4D284640F20C1201F044FAE1204102AA
:105B7000284601F0B7F9207850B1651C064CC1B237
:105B8000204601F0F3FA691C287800280D46F6D16A
:105B9000B0BDC046D9790030687A0030B0B504464F
:105BA000FFF774F9A100094A00245450092528B1CF
:105BB000016849698847002805DA4542FAF7F2FB8F
:105BC00005600020C4432046B0BDC04624320030EA
:105BD0000120EFF3108101400020401A4841704736
:105BE00080B500F0A5F9064801684A1C02D0491C9E
:105BF000016080BD03A010A13F2200F057FBC0460A
:105C000014790030637269746963616C5F736563F2
:105C100074696F6E5F7265656E7472616E63795FD1
:105C2000636F756E746572203C2055494E54333253
:105C30005F4D4158000000002E5C6D6265642D6F61
:105C4000735C706C6174666F726D5C736F75726398
:105C5000655C6D6265645F637269746963616C2E13
:105C6000630000000448016811B1491E016000D0C2
:105C7000704700F06BB9C046147900300120EFF393
:105C8000058101B90846704700B9FEE700F03CFB0A
:105C900080B510461A46FAF7C7FF002080BD000005
:105CA00010B561B102460B68002003E0934204D0B6
:105CB000CB691C315C1CF9D110BD084610BD02A097
:105CC00006A1172200F0F2FA6D6F6470726F705FB8
:105CD00074616220213D204E554C4C002E5C6D625B
:105CE00065642D6F735C746172676574735C544195
:105CF000524745545F4E55564F544F4E5C6E755F3C
:105D00006D6F647574696C2E630000000048704705
:105D1000E08C0110F0B581B00A4604460068411CD1
:105D200024D02272860840F2C0310E407D4971189D
:105D30000091617A062940D8C3B28F0001A5ED1900
:105D4000AF46C04600F014B800F01EB800F028B806
:105D500000F006B800F004B800F02FB800F033B837
:105D60000321042302B11946617226E001B0F0BD9F
:105D700001261D469E40002200983146FCF793FF05
:105D8000607A012803D008E001261D469E400222C9
:105D900000983146FCF787FF607A02282B4605D130
:105DA0000122114699400098FCF77DFF227A0321D9
:105DB000042002B101466172206801B0F0BC04BC4D
:105DC000964600F049BE0621002AF6D157497118BF
:105DD00040F2C0333C3382001A4001238B5006212D
:105DE000EBE7C046B0B504460160481C0BD00D4639
:105DF0000021284600F02EFE40F200202081E8B26B
:105E0000012181406160B0BD002200F001B80000B6
:105E100070B515460E460446FFF7E4FF701C1DD012
:105E20002068411C1BD00121002D0A4600D12A46C2
:105E300040F2C03340F2C0353C3586002E40800829
:105E400018403A4BC01882512046FFF763FF0021EB
:105E5000204670BC04BC964600F00AB870BD0248EB
:105E60000249282200F022FACE860110E6860110AF
:105E7000F0B581B004460068421C22D0850840F28B
:105E8000C0321540274BEB180093062931D8C6B213
:105E90008F0001A3DB199F4600F015B800F017B87A
:105EA00000F019B800F006B800F004B800F021B80E
:105EB00000F021B803292BD140F2003121810321C8
:105EC00029E001B0F0BD0121B140002206E001212E
:105ED000B140022202E001221146B1400098FCF7D5
:105EE000E2FE227A0321042002B101466172206899
:105EF00011E061720FE006216172237A5BB90B49F0
:105F000069183C32830013400122CA50062102E086
:105F100005492181042101B0F0BC04BC964600F083
:105F20009BBDC046004000500104000000480050E6
:105F3000EFF31080EFF3108172B60D490A7822B9A1
:105F400001220A7082430B480270704780B5EFF35C
:105F50001080C00707D0064800210170054800786E
:105F600000B162B680BD04A00AA1362200F09EF9FD
:105F7000F079003010790030216172655F696E74CC
:105F8000657272757074735F656E61626C656428AA
:105F9000290000002E5C6D6265642D6F735C686182
:105FA0006C5C6D6265645F637269746963616C5F88
:105FB00073656374696F6E5F6170692E63000000C2
:105FC00070B58EB014460D46064601A8001D30215E
:105FD000FAF7A9FE0395002E00DB184E019618482B
:105FE0003018032802D8686BEC6B00E001A8089019
:105FF0000294FFF7F5FD134801684A1C026049B995
:1060000001A811491CC81CC11CC81CC11CC81CC14A
:106010003CC83CC101A80D491CC81CC11CC81CC1FE
:106020001CC81CC13CC83CC10948016809B10748EB
:106030008847FFF717FE0EB070BDC0460101FF8014
:10604000C3FE007F1879003068790030A4790030F1
:106050001C790030F0B585B0044640683821415CB9
:1060600011B93A21405C08B105B0F0BD2068006864
:1060700080472068C06980470568002D4DD01F21EA
:10608000CAB201273B4693409D4204D0491E0026D8
:106090000A06F5D100E00E4640680290001F03900A
:1060A0001D2843D260680021019101604160206891
:1060B00040688047049464683B2166543A21019EFD
:1060C0006654A662E6622062A560F0430146029A29
:1060D000FAF7C3F9C1430720039A9040E1602061B9
:1060E000164A31463346FAF7D9F928187141401E4D
:1060F000B1412A463346FAF7E9F9A061E161266326
:1061000066632787049C204601F05EF9204605B0AF
:10611000F0BC02BC8E4600F04FBE00226846026012
:106120000748093016A1134600F054F900226846CA
:106130000260034803A1134600F04CF940420F00EF
:10614000050104805469636B6572206E756D62652C
:1061500072206F66206269742069732067726561BE
:10616000746572207468616E203332206F72206C07
:10617000657373207468616E2034206269747300E3
:106180005469636B6572206672657175656E6379BB
:10619000206973207A65726F0000000010B5FEF769
:1061A00075FE092430B10168C9698847002800DB01
:1061B00010BD4442FAF7F6F80460002010BD70B537
:1061C00014460D46FEF762FE092640B101680B69D0
:1061D000294622469847002800DB70BD4642FAF760
:1061E000E1F806600020C04370BD0000B0B517485C
:1061F000006C0820FAF7DAF8154908600120FAF770
:10620000D5F8144D286014A0FFF7A0FC1748FCF740
:106210005BFB1748FCF748FB000408D1FDF71AFDAB
:1062200028B1FEF75DF80446FDF71BFD2CB111A067
:10623000FFF78CFC134800F053F9286808B10021DF
:10624000017011A0FFF782FC0020B0BDB4800110E6
:10625000A07900300C3900300D0A4D62656420428F
:106260006F6F746C6F616465720D0A00EC31003001
:10627000415B0110626F6F74696E672E2E2E0D0ADE
:106280000D0A0000002402104661696C65642074E8
:106290006F206A756D7020746F206170706C696317
:1062A0006174696F6E210D0A0000000082B00B4618
:1062B0000146684602600248002200F08BF8C046A2
:1062C0004401FF80B0B584B00446002003900290E2
:1062D0000190FF259CB1102911D303A802A9FEF754
:1062E0001FF901060CD10299039801AA6B461A60A6
:1062F00010232246FDF75CFF0199102900D02846A3
:1063000040B204B0B0BD000086B0FFF769FC03A83E
:106310000A21FFF779FD002649E040F2C0343C3401
:1063200081002140800840F2C0321040264D2843B1
:10633000012201924250224F384601F0B3F90398EE
:10634000411C37D0810002942140800840F2C032C5
:106350001040284300224250384601F0A3F9761C31
:10636000042E24D300270398411C23D08100029ED1
:106370003140800840F2C0321040134C2043019A53
:106380004250104D284601F08DF90398411C11D060
:1063900081003140800840F2C03210402043002686
:1063A0004650284601F07EF97F1C042FDBD303986A
:1063B000411CB2D1054806492822FFF777FFC046A5
:1063C000F0490200801A060000480050CE860110F5
:1063D000E686011082B001930D460121094BD3E8F6
:1063E0004F7FC3E8441F39060AD17646029F114603
:1063F0007246FFF7E5FD284601993A4600F0F4FBA6
:1064000000F044F82079003083B080B581B003AF4C
:106410000EC703A9009100F01DF801B080BC01BCBB
:1064200003B00047B0B504460225002228462146A5
:1064300001F047F9FFF7D4FB2046FAF7D3FB0246F9
:106440002846214601F03DF9B0BC01BC8646FFF765
:1064500009BC000010B5A2B00B46024601A8842179
:10646000FAF7BCF80446842805D301A87F3005A1BB
:106470000522FAF7D9FB012C02DB01A8FFF7D2FFB6
:1064800022B010BD2E2E2E0A000000000D48012261
:10649000D0E84F1FC0E8432F002BF8D1C80705D024
:1064A000FFF79EFBBFF34F8F20BFFDE7FFF7E6FB33
:1064B00028B9FFF78DFB10B10120FFF7E5FBFFF7CF
:1064C00023FFC0469E7900307047000003480178E2
:1064D00001B1704701210170FDF728BAD879003069
:1064E000F0B5EFF3108172B6174A00211160CA436C
:1064F000164B174C174D8E003251725100263746FD
:10650000DE513F1D202FFBD12033491C0829F2D139
:1065100005214A0610490A604860104A8A60002234
:10652000CA601346CC18A2611B1D082BFAD10022A9
:106530000A6201684068002282F314888D4682F363
:1065400010880047F0BDC04610E000E000E400E025
:1065500080E100E080E200E004ED00E0FA050000E8
:10656000F0B5D6B00191009008300EA93CC83CC1EE
:106570003CC83CC13F20C0430690002011990A91BD
:10658000109907910F9D0E990B91139E14990D91DF
:10659000129F159909910D990B9C079B0F280D9639
:1065A00005900C950494039110D80199069A8918C6
:1065B00040240C5D240641254D5D2D042C194225F7
:1065C0004D5D2D0264194325495D1AE016A9069A0E
:1065D0008C5889184D6A64198D6B132638462F46DE
:1065E000F741AE0A7E401127FD4107467540641908
:1065F000496812250E46EE41CD0875400726F14147
:10660000694060180B9016ACA41820640C9C2546B9
:1066100004990D400C431C402C430B253E46EE4193
:10662000062508933846EF41774019250646029023
:10663000EE417E40244B9D182D6C099BED18AD1941
:106640000B9BEE180D9D039B5D4005405D4070194E
:1066500024180D250E46EE4102250F46EF417740E6
:1066600016250E46EE417E40A4190B940A9C27186D
:10667000121D0598401C0692C02A089A0A920C9A8C
:1066800007920D46029E099385D114463246129711
:1066900015930D98149013960F91109408981190DB
:1066A0000B990E91009DA8684018A8600EA8001DC7
:1066B0000C35002142586B589A186A50091D1C2944
:1066C000F8D1002056B0F0BD387A011021B10A4649
:1066D00002490B68002118477047C04658860110D0
:1066E000C046C046F0B581B00C46054607683F225B
:1066F0003946114006462836802070544B1CF0184D
:10670000382B04D83722511AFAF70BFB0BE0514013
:10671000FAF707FB28463146FFF722FF38213046BB
:10672000FAF701FB2F68780D64216854780B652116
:106730006854780966216854F800672168546868CD
:10674000410D6022A954410B6122A95441096222E2
:10675000A954790FC0004018632168542846314677
:10676000FFF7FEFEE87A207068896070A868000A6A
:10677000A070A868E070E87B2071E8896071E86823
:10678000000AA071E868E071E87C2072688A607293
:106790002869000AA0722869E072E87D2073E88AFF
:1067A00060736869000AA0736869E073E87E20740A
:1067B000688B6074A869000AA074A869E074E87F17
:1067C0002075E88B6075E869000AA075E869E075D6
:1067D0002320285C2076688C6076286A000AA076E0
:1067E000286AE076A86E48B92720285C2077E88CD4
:1067F0006077686A000AA077686AE077002001B0D5
:10680000F0BD10B16C21FFF761BF704780B56C21FE
:10681000FAF789FA80BD00000022026042608166BA
:1068200009B12C4A00E02A4A826009B12B4A00E0F3
:10683000294AC26009B12B4A00E0294A026109B124
:106840002A4A00E0284A426109B12A4A00E0284A5F
:10685000826109B1294A00E0274AC26109B1294A87
:1068600000E0274A026209B1284900E02649416256
:106870007047C046002202604260816609B1154B34
:1068800000E0134B836009B1144B00E0124BC3606E
:1068900009B1144B00E0124B036109B1134B00E046
:1068A000114B436109B1134B00E0114B836109B1F6
:1068B000124B00E0104BC36109B1124B00E0104BCA
:1068C000036209B1114900E00F4941621046704767
:1068D00067E6096AD89E05C185AE67BB07D57C36D9
:1068E00072F36E3C17DD70303AF54FA539590EF74B
:1068F0007F520E51310BC0FF8C68059B11155868F3
:10690000ABD9831FA78FF96419CDE05BA44FFABE02
:10691000C046C046F0B583B0002A44D014460E46A7
:10692000054601688A1802603F2308460293184012
:1069300040231F1A8A4202D26968491C69600021FB
:1069400090B1A74201D901460EE0294628310191B4
:10695000081831463A46FAF767F928460199FFF7D1
:10696000FFFDE41BF6190021402C15D3019102987C
:10697000C0432746403F38400090301840300290D6
:1069800028463146FFF7ECFD403C40363F2CF7D817
:1069900000983C1A0199029E2CB1681828303146A3
:1069A0002246FAF741F9002003B0F0BD0648002165
:1069B000017000F09DBDC04680B500F0ADFD0248FD
:1069C0000121017080BDC046F4380030F0B585B0BB
:1069D0000D460646FDF704FE0446002835DB002779
:1069E000049702A83146FEF75FFBFEF74AFBF8B1B9
:1069F00002A8FEF74BFB20B102A8FEF734FB04907F
:106A000020E002A8FEF720FB90B1064602A8FEF7A0
:106A100049FB024630688068019004A930462B4645
:106A2000019DA84768B14542F9F7BCFC056003E049
:106A3000F9F7B8FC13210160A00005490F50FC4391
:106A400003E00498A100024A5050204605B0F0BD72
:106A50002432003000F0D6BE80B5421C12D0C91ED0
:106A6000CAB2032A0DD8C3B201219940800840F26E
:106A7000C03303400648181880BC08BC9E46FCF78B
:106A8000FEB880BD03A008A12722FFF70FFCC04677
:106A90000040005070696E20213D202850696E4EE4
:106AA000616D65294E4300002E5C6D6265642D6F3B
:106AB000735C746172676574735C544152474554EA
:106AC0005F4E55564F544F4E5C5441524745545FAC
:106AD0004D323335315C70696E6D61702E6300002C
:106AE00080B582B0024688420BD0501C08D0481CAA
:106AF00007D0002368460360034804A1FFF76AFC3F
:106B00000A46104602B080BD3001018070696E6D8A
:106B10006170206D69732D6D617463680000000001
:106B200010B582B002460120C343581C541C14D037
:106B30000868441C06D00C3190420AD008680C3119
:106B4000441CF9D1002368460360054805A1FFF7FE
:106B500041FC98000858411CF4D002B010BDC0465A
:106B60003001018070696E6D6170206E6F742066F7
:106B70006F756E6420666F722070657269706865EB
:106B800072616C0010B582B00446401C1DD00868CC
:106B9000421C06D00831A0420BD048680C31421C80
:106BA000F9D100236846036009480AA12246FFF78D
:106BB00011FC09682046FFF74DFF0021204602B076
:106BC00010BC04BC9646FFF747BF02B010BDC046DC
:106BD00030010180636F756C64206E6F7420706982
:106BE0006E6F757400000000F0B581B000920D4624
:106BF0000646032040073E4C21680A4602404F42A9
:106C0000824200D08FB2080CC3B23A483A46FFF72E
:106C1000FBFB39483818132845D8810001A25118C8
:106C20008F46C04600F026B800F027B800F028B81C
:106C300000F029B800F02AB800F02BB800F02CB80A
:106C400000F02DB800F02FB800F02DB800F02BB8F0
:106C500000F029B800F027B800F025B800F023B8FC
:106C600000F021B800F01FB800F01DB800F01BB80C
:106C700000F03AB8A168474813E0A16841A010E0CD
:106C8000A1683CA00DE0A16835A00AE0A1682FA092
:106C900007E0A16824A004E0A16827A001E0A168A2
:106CA0001BA0FFF7B1FB3046FFF7BCFB61683A4819
:106CB000FFF7AAFB4DB139A0FFF7B4FB2846FFF759
:106CC000B1FB38A00099FFF79FFBA1683648FFF79A
:106CD0009BFB21683548FFF797FB354801B0F0BCB6
:106CE00002BC8E46FFF790BB04A0FFF78DFBDAE7EE
:106CF000A4790030AB870110CFFEFFFF41737365AD
:106D00007274696F6E206661696C65643A20000078
:106D10004D65737361676551756575653A203078A7
:106D200025582C200000000054696D65723A20300F
:106D30007825582C200000004576656E74466C61FD
:106D400067733A20307825582C2000004D656D6F10
:106D50007279506F6F6C3A20307825582C200000E3
:106D600053656D6170686F72653A20307825582CD4
:106D7000200000004D757465783A20307825582C35
:106D8000200000005468726561643A20307825580C
:106D90002C20000096870110658801100A46696C56
:106DA000653A20002B25640052880110FC870110F1
:106DB0007C87011070470000F0B581B0044646683A
:106DC0003A20305C10B93920305C08B101B0F0BD18
:106DD000204600F0F9FA67687968E1B103C93B6BB6
:106DE0007A6B1D1A15468D4148D2C01A91413D69F2
:106DF000BA69FB69121A8B4128D3BA68264B9A42AA
:106E000021D03B23FB5C93B11A46F9F726FB002304
:106E1000224A801813E0306AF1683269101808407D
:106E20002168096901B0F0BC04BC964608470023FC
:106E30000093009BF9F732FB184A8018009B5941D8
:106E4000154AF9F743FB854200D30546386A4019D5
:106E5000FD680540306A854217D0206801692846E0
:106E60008847206840688047316A8D4202D9A8422D
:106E700002D303E0A842A9D38842A7D22068406980
:106E800001B0F0BC02BC8E46004705A00DA140F247
:106E90001B12FFF70BFAC04640420F003F420F00A3
:106EA0006D617463685F7469636B20213D20717547
:106EB0006575652D3E7469636B5F6C6173745F7299
:106EC000656164002E5C6D6265642D6F735C686142
:106ED0006C5C6D6265645F7469636B65725F617041
:106EE000692E63000368B14A1A409369DB00FCD540
:106EF00041611046FCF79CBD70B582B00446056840
:106F0000254828408569ED00FCD54D1F042D2ED263
:106F1000052A32D25D1E022D36D218340EC400244A
:106F2000052908D0062901D1012404E00224032503
:106F3000072900D02C4602211143082503290CD132
:106F40009A1E00218B1A53419A006B461A60224602
:106F50002B46FCF7DBFD02B070BD18250026042A85
:106F6000294600D03146022AEAD00D46E8E70B4810
:106F70000B4940F25F12FFF799F940F25F10421C93
:106F800008480749FFF792F940F25F10821C06A0FB
:106F90000349FFF78BF9C046E0FF0FFF5C89011042
:106FA000C8890110D88801102873746F705F6269F6
:106FB0007473203D3D203129207C7C202873746F20
:106FC000705F62697473203D3D203229000000002B
:106FD00001460068754A024090694004FCD410687C
:106FE0003423CB5C11210B4202D053680B43536016
:106FF0007047C046F0B581B017460D460446FFF70E
:1070000065FA44492846FFF78BFD06464249384653
:10701000FFF786FD01463046FFF762FD2060411C08
:1070200062D03E49FEF73CFE002862D0226801682B
:10703000914263D13B46009087690020C64365605A
:1070400028461D46A360E66026613249FFF79AFD97
:1070500031492846FFF796FD386808BB009D2A1D78
:1070600007CA00F087FB686800F08AFB286900F017
:107070007BFB22682C4810402C4B8169C900FCD551
:10708000E12149029A4201D042F280516161FCF74C
:10709000CFFC0821002201232046FFF72DFF38688E
:1070A000401C386039690022226361622287E663EE
:1070B000266462641E498C42009A07D120681B49ED
:1070C000884220D11C4801210160386850B1134822
:1070D000101A8010194941430120884018490A6854
:1070E00002430A6001B0F0BD17A00E49C322FFF7AA
:1070F000DDF814480B49C622FFF7D8F808480949BB
:10710000C722FFF7D3F80B48064940F20712FFF7F2
:10711000CDF8C046747E0110347C01101C8C011027
:10712000038A0110C8890110E0FF0FFF000007501B
:10713000F4790030A9890110DC7A0030B76DDBB634
:10714000E47A00306186011028696E74296F626AE2
:107150002D3E73657269616C2E7561727420213DDC
:10716000204E4300CA684968FFF744BF0368954A48
:107170001A4093691B02FCD411603421405C8007E3
:1071800003D55068022101435160704700688D4962
:1071900001408869810B0120884370470068894954
:1071A00001408869C10D012088437047E0FF0FFF4F
:1071B00070B50446FEF714FD2068C068804760681B
:1071C0003A21415C09BB39210122425441683930DE
:1071D000B1B1204600F0F8F86068026B436B41687B
:1071E0000D684E68521BB34109D3CA6842600368F8
:1071F0001BB18868984760684268002AE9D1393035
:10720000002101702046FFF7D7FD70BC01BC864607
:10721000FEF728BD80B500F001F880BDB0B504468A
:10722000FEF718FFFEF7DCFC204600F0CDF86068A2
:10723000046B456BFEF716FD20462946B0BD0000E5
:10724000A2480121016000F0FBB9C0460A4840682D
:1072500000F08CB810B508484468606B11210842F2
:1072600002D0E06C8047606B800700D410BDA06C3A
:1072700010BC02BC8E4600476C3200300A484068A1
:1072800000F074B810B508484468606B11210842DA
:1072900002D0E06C8047606B800700D410BDA06C0A
:1072A00010BC02BC8E460047883200300A48406855
:1072B00000F05CB810B508484468606B11210842C2
:1072C00002D0E06C8047606B800700D410BDA06CDA
:1072D00010BC02BC8E460047A43200300A48406809
:1072E00000F044B810B508484468606B11210842AA
:1072F00002D0E06C8047606B800700D410BDA06CAA
:1073000010BC02BC8E460047C03200300A484068BC
:1073100000F02CB810B508484468606B1121084291
:1073200002D0E06C8047606B800700D410BDA06C79
:1073300010BC02BC8E460047DC3200300A48406870
:1073400000F014B810B508484468606B1121084279
:1073500002D0E06C8047606B800700D410BDA06C49
:1073600010BC02BC8E460047F8320030B0B504466F
:107370000068144D0540E86941F2001108420CD044
:107380006968112081436960A26A32B13421615C6D
:10739000014202D0E06A00219047E86980050CD5DF
:1073A0006868022188436860A26A32B13420205C98
:1073B000800702D5E06A01219047E869E861A86981
:1073C000A861B0BDE0FF0FFFF0B587B00446476885
:1073D0003A20385C002873D1206840688047616893
:1073E000096A88426CD0396A3862401AB968FD6807
:1073F00005400022754881425CD00691734A002105
:10740000284604910B46F9F749F80C463B217E5C6F
:10741000BD6AF96A3B4628330593002E0391029515
:107420000190214619D03246F9F727F80546009118
:107430003246F9F712F8019A101A8C410299401855
:1074400005990860039A54414C60069BC11A214675
:10745000049A914125D2009A2CE0069A049E334664
:10746000F9F734F805460091069A3346F9F716F80D
:107470003346009A019E301A8C41029940180599B2
:107480000860039E7441069E4C60811B2146994111
:1074900010D3801B059908609C414C606D1C5A41BB
:1074A00008E0C01A0599086094414C606D1C009872
:1074B00050410246386B40193863786B504178630D
:1074C00007B0F0BD01480121016070470810055068
:1074D0003A4804210160BFF34F8FBFF36F8F7047AD
:1074E0000248042101606E480160704704E200E038
:1074F00080B5324804210160BFF34F8FBFF36F8F17
:107500002F4800F025F958480021018080BDC04671
:10751000004870470C8D0110B0B52748018839B17B
:10752000264804210160BFF34F8FBFF36F8FB0BDBA
:10753000012505806904224C0022204600F01AF93A
:10754000204600F01DF91F4800F00EF91E4C2046A1
:10755000FCF710FA1D4AB0FBF2F3591E802920D225
:107560005A43801A22D10320C006014321604B48B0
:10757000606031480068C821304A42500F480421F9
:107580000160BFF34F8FBFF36F8F6807216801431E
:107590002160A80721680143216020688001FCD593
:1075A000B0BD0BA019496922FEF780FE18A017494B
:1075B0006A22FEF77BFEC046E07A003084E100E0FC
:1075C0000400005F040000040010055040420F005A
:1075D000287072657363616C655F74696D65722094
:1075E000213D202875696E7433325F7429202D3156
:1075F00029202626207072657363616C655F74694B
:107600006D6572203C3D2031323700002E8A01101A
:1076100028636C6B5F74696D65722025204E555F21
:10762000544D52434C4B5F5045525F5345432920C4
:107630003D3D20300000000008ED00E041720110E7
:107640000248016809B102480847704768320030B3
:10765000E08C011080B50448008808B9FFF75CFF92
:107660000248006880BDC046E07A00300C1005502A
:10767000084901224A60084B04221A6002230228AA
:1076800000D81846054B984200D3184608600448B5
:10769000026070470410055084E200E0FFFFFF0025
:1076A00004E100E070B50446FEF730FB0546FFF745
:1076B000B1FD06462846FFF7ADFD801BA042F9D379
:1076C00070BD70B514460D46FDF7E0FB092640B1CC
:1076D0000168CB68294622469847002800DB70BD28
:1076E0004642F8F75FFE06600020C04370BD000010
:1076F00003B40148019001BDB1D0000003B40148BA
:10770000019001BD79D0000003B40148019001BD92
:1077100081D0000003B40148019001BD71D0000088
:1077200003B40148019001BD99D0000003B40148A1
:10773000019001BDA1D0000003B40148019001BD3A
:10774000A9D0000003B40148019001BD91D0000010
:1077500003B40148019001BDC1D0000003B4014849
:10776000019001BDF9D0000003B40148019001BDB2
:10777000F1D0000003B40148019001BDE1D0000048
:1077800003B40148019001BDC9D0000003B4014811
:10779000019001BDE9D0000003B40148019001BD92
:1077A00061D0000003B40148019001BD41D0000048
:1077B00003B40148019001BD31D0000003B4014879
:1077C000019001BD51D0000003B40148019001BDFA
:1077D00039D0000003B40148019001BD59D0000028
:1077E00003B40148019001BD49D0000003B4014831
:1077F000019001BD29D0000003B40148019001BDF2
:1078000069D0000003B40148019001BD01D100001E
:10781000F0B4040C8BB2264682B25E431046584345
:107820000D0C370C360400218019164679416E4341
:10783000370C36048019264679416E438919F0BC0D
:10784000704700004900CA020243100000D0042023
:107850004A0D01D001221043044A490D914201D141
:1078600002210843012800D105207047FF070000CE
:1078700030380A2801D2012070470020704710B527
:107880008A68002A02DCF9F79DFC10BD521E8A604E
:107890004A68C0B2531C4B60107010BD10B500296F
:1078A0000AD00878002807D005487844F9F73EFA4E
:1078B000002801D0002010BD0248784410BD00000F
:1078C0008A1400008214000010B500290AD008783C
:1078D000002807D005487844F9F728FA002801D095
:1078E000002010BD0248784410BD00006E15000055
:1078F0006615000003B402487844844603BC604720
:1079000055A1FFFF03B402487844844603BC604796
:10791000BDA3FFFF30313233343536373839414279
:1079200043444546403058003031323334353637E1
:10793000383961626364656640307800040000088D
:107940000000000000000002000100001000000024
:10795000000000000000000030313233343536378B
:10796000383961626364656678700030313233346F
:1079700035363738394142434445465850000000B7
:1079800002400000000000A00000000005400000D0
:10799000000000C8000000000C4000000000409CF7
:1079A00000000000194000000020BCBE00000000E4
:1079B00034400000BFC91B8E00000004B540000029
:1079C000504BCFD06607E2CF010000006C410000B1
:1079D0003E8251AADFEEA73401000000D942000028
:1079E000DCB5A0E23A301F97FFFFFFFFB44500006F
:1079F000FD25A0C8E9A3C14FFFFFFFFFFF3F000027
:107A00000000008000000000FF3F00000000008038
:107A1000000000002000000020000000688A011023
:107A2000004000000000000010390030004000005D
:107A30000000000010390030982F8A4291443771BD
:107A4000CFFBC0B5A5DBB5E95BC25639F111F159E1
:107A5000A4823F92D55E1CAB98AA07D8015B831223
:107A6000BE853124C37D0C55745DBE72FEB1DE80CF
:107A7000A706DC9B74F19BC1C1699BE48647BEEFFE
:107A8000C69DC10FCCA10C246F2CE92DAA84744A89
:107A9000DCA9B05CDA88F97652513E986DC631A8FF
:107AA000C82703B0C77F59BFF30BE0C64791A7D5DE
:107AB0005163CA0667292914850AB72738211B2E66
:107AC000FC6D2C4D130D385354730A65BB0A6A764E
:107AD0002EC9C281852C7292A1E8BFA24B661AA85A
:107AE000708B4BC2A3516CC719E892D1240699D66A
:107AF00085350EF470A06A1016C1A419086C371EE3
:107B00004C774827B5BCB034B30C1C394AAAD84EC0
:107B10004FCA9C5BF36F2E68EE828F746F63A578FB
:107B20001478C8840802C78CFAFFBE90EB6C50A48E
:107B3000F7A3F9BEF27871C60C01000000D0005026
:107B4000000009000D03000000D0005000003000CC
:107B5000FFFFFFFFFFFFFFFF00000000010100002B
:107B600000D00050300000000604000000D000509B
:107B700000000003FFFFFFFFFFFFFFFF000000000A
:107B80000001000000D000500300000007040000C6
:107B900000D0005000000030FFFFFFFFFFFFFFFF9D
:107BA000000000000201000000D0005000030000AF
:107BB0000204000000D0005000030000FFFFFFFFA0
:107BC000FFFFFFFF000000000301000000D0005095
:107BD000003000000304000000D00050003000001E
:107BE000FFFFFFFFFFFFFFFF000000000401000098
:107BF00000D00050000003000404000000D000503A
:107C000000000300FFFFFFFFFFFFFFFF0000000079
:107C10000501000000D00050000030000504000005
:107C200000D0005000003000FFFFFFFFFFFFFFFF0C
:107C300000000000000000000000075007000000E6
:107C400002000000001017500008000002100100A0
:107C500000101750000800000200000000404750CC
:107C600000070000024001000040475000070000EC
:107C700004000000005057500000080006000000FB
:107C80000000075000000007080000000010175017
:107C9000070000000D0000000040475000003000C9
:107CA0000F0000000000075000000030000100003D
:107CB00000202750070000000201000000101750AC
:107CC00000060000040100000050575000000700AB
:107CD0000601000000101750000000060801000017
:107CE00000000750050000000A0100000040475056
:107CF000000600000C010000000007500000060014
:107D00000E010000003037500000000700020000A4
:107D10000020275008000000020200000030375009
:107D2000000B0000040200000020275000000800A3
:107D30000422010000202750000008000402000077
:107D40000040475000000B00044201000040475033
:107D500000000B0006020000004047500000000534
:107D6000080200000010175008000000090200007F
:107D700000303750700000000B0200000000075078
:107D80000030000000030000003037500500000004
:107D90000203000000000750000900000603000075
:107DA00000101750000000030A03000000101750D5
:107DB000000300000C030000002027500000070013
:107DC00000040000003037500700000006040000E7
:107DD0000050575000000008090400000020275000
:107DE000700000000B0400000030375000700000ED
:107DF0000F040000002027500000003001050000A3
:107E0000001017502000000002050000000007507D
:107E1000000300000505000000202750000020009E
:107E2000060500000040475000000006090700005A
:107E300000101750A00000000B07000000000750C2
:107E4000008000000B0701000000075000800000C8
:107E50000B07000000404750007000000B47010076
:107E60000040475000700000FFFFFFFFFFFFFFFFD3
:107E7000000000000100000000000750700000003A
:107E800003000000001017500080000003100100E4
:107E90000010175000800000030000000040475011
:107EA00000700000034001000040475000700000D7
:107EB000050000000050575000008000070000003F
:107EC000000007500000007009000000001017506B
:107ED000700000000C00000000404750000003004C
:107EE0000E00000000000750000000030101000028
:107EF0000020275070000000030100000010175000
:107F000000600000050100000050575000007000A4
:107F10000701000000101750000000600901000078
:107F200000000750500000000B01000000404750C7
:107F3000006000000D01000000000750000060001C
:107F40000F010000003037500000007001020000F7
:107F5000002027508000000003020000003037504E
:107F600000B0000005020000002027500000800043
:107F700005220100002027500000800005020000BB
:107F8000004047500000B00005420100004047504B
:107F90000000B00007020000004047500000005001
:107FA0000A02000000303750000700000C020000F9
:107FB00000000750000003000D02000000202750C1
:107FC0000000700001030000003037505000000036
:107FD00003030000000007500090000007030000AA
:107FE00000101750000000300B0300000010175065
:107FF0000030000001040000003037507000000025
:1080000007040000005057500000008008040000E2
:1080100000202750070000000A04000000303750FD
:10802000000700000D040000001017500000800041
:108030000E0400000020275000000003000500008F
:108040000010175002000000030500000000075058
:10805000003000000405000000202750000002004E
:1080600007050000004047500000006008070000BE
:10807000001017500A0000000A0700000000075017
:10808000000800000A070100000007500008000077
:108090000A07000000404750000700000A4701009F
:1080A0000040475000070000FFFFFFFFFFFFFFFFFA
:1080B00000000000000000000000000000000000C0
:1080C00000000000000000000000000000000000B0
:1080D00000000000000000000000000000000000A0
:1080E0000000000000000000000000000000000090
:1080F000000000000000000000D0005006FF430711
:108100000000200000000001060000004000000008
:1081100000000000FFFFFFFF000000000000000063
:10812000000000000000000000000000000000004F
:10813000554601105D460110654601106D4601105F
:10814000754601107D460110854601108D460110CF
:1081500000000000B71DC1046E3B8209D926430D03
:10816000DC7604136B6BC517B24D861A0550471E9B
:10817000B8ED08260FF0C922D6D68A2F61CB4B2B3B
:10818000649B0C35D386CD310AA08E3CBDBD4F38E3
:1081900070DB114CC7C6D0481EE09345A9FD524183
:1081A000ACAD155F1BB0D45BC2969756758B56521B
:1081B000C836196A7F2BD86EA60D9B6311105A67BB
:1081C00014401D79A35DDC7D7A7B9F70CD665E7463
:1081D000E0B6239857ABE29C8E8DA19139906095C3
:1081E0003CC0278B8BDDE68F52FBA582E5E66486DB
:1081F000585B2BBEEF46EABA3660A9B7817D68B3FB
:10820000842D2FAD3330EEA9EA16ADA45D0B6CA022
:10821000906D32D42770F3D0FE56B0DD494B71D942
:108220004C1B36C7FB06F7C32220B4CE953D75CA5A
:1082300028803AF29F9DFBF646BBB8FBF1A679FF7A
:10824000F4F63EE143EBFFE59ACDBCE82DD07DECA2
:1082500077708634C06D4730194B043DAE56C53932
:10826000AB0682271C1B4323C53D002E7220C12A6A
:10827000CF9D8E1278804F16A1A60C1B16BBCD1F6A
:1082800013EB8A01A4F64B057DD00808CACDC90CB2
:1082900007AB9778B0B6567C69901571DE8DD475B2
:1082A000DBDD936B6CC0526FB5E6116202FBD066EA
:1082B000BF469F5E085B5E5AD17D1D576660DC53EA
:1082C00063309B4DD42D5A490D0B1944BA16D84032
:1082D00097C6A5AC20DB64A8F9FD27A54EE0E6A172
:1082E0004BB0A1BFFCAD60BB258B23B69296E2B22A
:1082F0002F2BAD8A98366C8E41102F83F60DEE87AA
:10830000F35DA9994440689D9D662B902A7BEA9471
:10831000E71DB4E0500075E4892636E93E3BF7EDF1
:108320003B6BB0F38C7671F7555032FAE24DF3FEA9
:108330005FF0BCC6E8ED7DC231CB3ECF86D6FFCB29
:108340008386B8D5349B79D1EDBD3ADC5AA0FBD8F1
:10835000EEE00C6959FDCD6D80DB8E6037C64F6451
:108360003296087A858BC97E5CAD8A73EBB04B7709
:10837000560D044FE110C54B383686468F2B4742C9
:108380008A7B005C3D66C158E4408255535D435191
:108390009E3B1D252926DC21F0009F2C471D5E28D1
:1083A000424D1936F550D8322C769B3F9B6B5A3B89
:1083B00026D6150391CBD40748ED970AFFF0560E49
:1083C000FAA011104DBDD014949B93192386521D11
:1083D0000E562FF1B94BEEF5606DADF8D7706CFC11
:1083E000D2202BE2653DEAE6BC1BA9EB0B0668EF49
:1083F000B6BB27D701A6E6D3D880A5DE6F9D64DA89
:108400006ACD23C4DDD0E2C004F6A1CDB3EB60C9D0
:108410007E8D3EBDC990FFB910B6BCB4A7AB7DB090
:10842000A2FB3AAE15E6FBAACCC0B8A77BDD79A3C8
:10843000C660369B717DF79FA85BB4921F46759608
:108440001A163288AD0BF38C742DB081C330718550
:1084500099908A5D2E8D4B59F7AB085440B6C950A0
:1084600045E68E4EF2FB4F4A2BDD0C479CC0CD43B8
:10847000217D827B9660437F4F460072F85BC17618
:10848000FD0B86684A16476C93300461242DC56540
:10849000E94B9B115E565A1587701918306DD81C20
:1084A000353D9F0282205E065B061D0BEC1BDC0F38
:1084B00051A69337E6BB52333F9D113E8880D03A98
:1084C0008DD097243ACD5620E3EB152D54F6D429C0
:1084D0007926A9C5CE3B68C1171D2BCCA000EAC8E0
:1084E000A550ADD6124D6CD2CB6B2FDF7C76EEDB78
:1084F000C1CBA1E376D660E7AFF023EA18EDE2EE58
:108500001DBDA5F0AAA064F4738627F9C49BE6FDFF
:1085100009FDB889BEE0798D67C63A80D0DBFB845F
:10852000D58BBC9A62967D9EBBB03E930CADFF97F7
:10853000B110B0AF060D71ABDF2B32A66836F3A2D7
:108540006D66B4BCDA7B75B8035D36B5B440F7B17F
:1085500000000000000000003B4E0110E147011048
:1085600061470110854701107547011081470110CF
:108570000F4E0110A9470110134E01102B4E011090
:108580007B470110354E0110234E01101D4E011086
:10859000094E0110F74D0110C1520110F14D0110AB
:1085A000034E0110DD510110294E011000000000A2
:1085B00000000000C54D0110B54D0110E547011048
:1085C000114A0110854E011015490110414A011050
:1085D000054A0110894E0110795201109152011083
:1085E00081520110895201109953011099520110C2
:1085F000C55201109F53011033530110B5520110A1
:10860000014A01100000000000000000C54F0110E9
:10861000C14F01106D4F0110FFFFFFFF0D01000062
:10862000FFFFFFFF0C010000FFFFFFFF0000000045
:108630002F737464657272002F737464696E002FF7
:108640007374646F75740000001BB70000000000B5
:1086500000800000001BB700AB0C01105F73646862
:108660005F6D6F64696E697420213D204E554C4CDE
:10867000002E5C647269766572735C73746F7261EC
:1086800067655C434F4D504F4E454E545F4E5553BA
:10869000445C4E755344426C6F636B44657669630A
:1086A000652E6370700063726320213D204E554C2F
:1086B0004C002E2F6D6265642D6F732F6472697686
:1086C0006572735C4D6265644352432E68006F624D
:1086D0006A2D3E70696E20213D202850696E4E61E2
:1086E0006D65294E43002E2F6D6265642D6F732FCB
:1086F000746172676574732F5441524745545F4EDD
:1087000055564F544F4E2F5441524745545F4D32AA
:108710003335312F6770696F5F6F626A6563742EDE
:10872000680052616E206F7574206F662043546834
:10873000756E6B20656E74726965732E20496E6369
:108740007265617365204D4245445F434F4E465FFD
:10875000504C4154464F524D5F435448554E4B5F29
:10876000434F554E545F4D415820746F20666978D1
:108770002074686973206572726F72000A2D2D2053
:108780004D6265644F53204572726F7220496E6668
:108790006F202D2D0A004B65726E656C204572723C
:1087A0006F723A20307825582C20000A0A2B2B2093
:1087B0004D6265644F53204572726F7220496E6638
:1087C0006F202B2B0A4572726F722053746174757F
:1087D000733A203078255820436F64653A20256429
:1087E000204D6F64756C653A2025640A4572726F7E
:1087F00072204D6573736167653A20000A466F7297
:10880000206D6F726520696E666F2C2076697369C2
:10881000743A2068747470733A2F2F6D6265642EF9
:10882000636F6D2F732F6572726F723F6572726F17
:10883000723D307825303858267467743D4E555F48
:1088400050464D5F4D323335315F4E5053415F4E90
:1088500053000A4572726F722056616C75653A203A
:1088600030782558000A4C6F636174696F6E3A2046
:108870003078255800286775617264202620435897
:10888000415F47554152445F4D41534B29203D3D87
:10889000204358415F47554152445F494E49545F18
:1088A000494E5F50524F4752455353002E5C6D6204
:1088B00065642D6F735C706C6174666F726D5C7350
:1088C0006F757263655C6D6265645F726574617219
:1088D0006765742E63707000287061726974792006
:1088E0003D3D205061726974794E6F6E6529207C20
:1088F0007C2028706172697479203D3D205061723E
:108900006974794F646429207C7C202870617269C5
:108910007479203D3D205061726974794576656EA9
:1089200029207C7C2028706172697479203D3D206B
:10893000506172697479466F726365643129207C75
:108940007C2028706172697479203D3D20506172ED
:10895000697479466F7263656430290028646174B4
:10896000615F62697473203D3D203529207C7C2045
:1089700028646174615F62697473203D3D2036290B
:10898000207C7C2028646174615F62697473203D7F
:108990003D203729207C7C2028646174615F6269F6
:1089A0007473203D3D203829006F626A2D3E736547
:1089B0007269616C2E75617274203D3D2053544480
:1089C000494F5F55415254002E5C6D6265642D6FB6
:1089D000735C746172676574735C544152474554AB
:1089E0005F4E55564F544F4E5C5441524745545F6D
:1089F0004D323335315C73657269616C5F617069EA
:108A00002E63006D6F64696E69742D3E6D6F646EC8
:108A1000616D65203D3D2028696E7429206F626A72
:108A20002D3E73657269616C2E75617274002E5CE7
:108A30006D6265642D6F735C746172676574735CDD
:108A40005441524745545F4E55564F544F4E5C5417
:108A500041524745545F4D323335315C75735F7415
:108A600069636B65722E630053746F72616765454D
:108A70006E63323536484D414353484132353653A3
:108A800049474E4154555245005B455252205D20A6
:108A90004153534552540D0A005B444247205D2028
:108AA0004669726D776172652073697A6520726FAD
:108AB000756E64656420757020746F20746865201D
:108AC0006E65617265737420736563746F72206282
:108AD0006F756E64617279206973206C617267656D
:108AE00072207468616E20746865206D6178696DAC
:108AF000756D206170706C69636174696F6E20734D
:108B0000697A650D0A005B444247205D2046697220
:108B10006D77617265207570646174652066616946
:108B20006C65640D0A0055706461746520696D613F
:108B3000676520696E74656772697479206368651A
:108B4000636B206661696C65640D0A005B44424793
:108B5000205D204E657720616374697665206669C3
:108B6000726D776172652069732076616C69640D3E
:108B70000A005B455252205D20416374697665208E
:108B80006669726D7761726520696E76616C696481
:108B90000D0A004E6F2055706461746520696D6127
:108BA00067650D0A0055706461746520696D6167C1
:108BB0006520746F6F206C617267650D0A005B44FD
:108BC0004247205D2055706461746520616374695B
:108BD0007665206669726D776172650D0A005B4487
:108BE0004247205D20416374697665206669726D35
:108BF000776172652075702D746F2D646174650DD9
:108C00000A0055706461746520696D61676520694B
:108C100073206F6C6465720D0A000000000007503D
:108C2000103D805700000003000000001000000409
:108C3000240000006C32003000101750913DA05706
:108C40000000000C000000001100000425000000DE
:108C50008832003000202750123C8C77000000033F
:108C6000000000001200000430000000A4320030B8
:108C700000303750933CAC770000000C000000003F
:108C80001300000431000000C032003000404750A3
:108C9000143DCC77000000300000000014000004F8
:108CA0004A000000DC32003000505750953DEC7710
:108CB000000000C000000000150000044B00000090
:108CC000F8320030FFFFFFFF00000000000000004E
:108CD0000000000000000000000000000000000094
:108CE000E88C011028790030B9690110557601101F
:108CF000D1740110C574011071760110E174011076
:108D0000AD690110117501100000000040420F0014
:108D100018000000648E0110E031003034010000C2
:108D2000D4270110D08E011014330030D447000036
:108D30001C0201101001000043000000F8FFFFFFBB
:108D4000004040404040404040404141414141405E
:108D50004040404040404040404040404040404013
:108D600040050202020202020202020202020202A2
:108D700002202020202020202020200202020202A7
:108D800002029090909090901010101010101010FF
:108D9000101010101010101010101010020202020B
:108DA000020288888888888808080808080808084F
:108DB000080808080808080808080808020202024B
:108DC0004000000000000000000000000000000063
:108DD0000000000000000000000000000000000093
:108DE0000000000000000000000000000000000083
:108DF0000000000000000000000000000000000073
:108E00000000000000000000000000000000000062
:108E10000000000000000000000000000000000052
:108E20000000000000000000000000000000000042
:108E30000000000000000000000000000000000032
:108E4000000000001C00000043000000F8FFFFFFCE
:108E50000C0000000E0000000F0000002E000000BB
:108E6000E5ADFFFFC10514652801104BDD29185E33
:108E7000652A0110050C42302C6CDC02049AFF01BB
:108E8000013429388BB1717C290929041E4D7201E6
:108E9000105504A30405691C1A7D181A85040B10CB
:108EA00006071C1AAD181AB5040B1008091C1ADDA8
:108EB000181AE5040B100A0B1C1E0D730110150483
:108EC0000B100C0D1C1A3D181A4504230E0F000040
:04000005100101D90C
:00000001FF
